:020000040000FA
:04000000C1EF04F058
:04000800F7EF27F0F7
:0800180056EF28F00F0B176EE4
:10002000000EF76E360EF66E1750F626D8B0F72A89
:100030000800F55012003031323334353637383954
:10004000414243444546536A3AC145F03BC146F0FC
:100050003CC147F03DC148F03EC149F041C14AF0C2
:1000600042C14BF043C14CF044C14DF045C14EF08C
:1000700046EC31F049AE0AD03E0E496E4C0E486E49
:10008000CC0E476ECC0E466ECD0E456E45C046F189
:1000900046C047F147C048F148C049F149C04AF15C
:1000A00049EC33F033EC2EF026C0A2F027C0A3F0C9
:1000B0001200536A79EC2CF064C030F065C031F066
:1000C000FCEC2EF073EC30F03F0E4E6EC80E4D6E11
:1000D0004A6A4B6A4C6A89EC30F045C074F146C0FC
:1000E00075F147C076F148C077F149C078F1A4ECCA
:1000F0002EF01200536A79EC2CF063C030F0FCEC67
:100100002EF073EC30F03E0E4E6E4A6A4B6A4C6A2B
:100110004D6A89EC30F045C06FF146C070F147C0C0
:1001200071F148C072F149C073F1A4EC2EF01200D5
:10013000536A3EC130F030AE06D0456A466A476A1F
:10014000486A496A19D046C145F047C146F048C1DE
:1001500047F049C148F04AC149F049AE0BD0420EC0
:10016000496EC70E486EFA0E476EE10E466E480E97
:10017000456E02D043EC38F045C09DF046C09EF07D
:1001800047C09FF048C0A0F049C0A1F049EC33F04F
:1001900019EC2EF026C0A4F027C0A5F01200410EE5
:1001A0004E6EF90E4D6E020E4C6E260E4B6E810E8B
:1001B0004A6E1200536AA9C030F0ECEC00F026C081
:1001C000ABF027C0ACF0AAC030F0ECEC00F026C0D9
:1001D000ADF027C0AEF01200536AF4EC2EF073ECD1
:1001E00030F0CFEC00F046EC31F05AC14AF05BC180
:1001F0004BF05CC14CF05DC14DF05EC14EF046EC81
:1002000031F055C14AF056C14BF057C14CF058C1BE
:100210004DF059C14EF009EC31F019EC2EF01200FE
:1002200079EC2CF096C030F097C031F055C14BF10D
:1002300056C14CF157C14DF158C14EF159C14FF162
:100240005AC150F15BC151F15CC152F15DC153F132
:100250005EC154F166EC01F045C03AF146C03BF195
:1002600047C03CF148C03DF149C03EF149EC33F094
:1002700019EC2EF026C03FF127C040F1120079ECB6
:100280002CF098C030F099C031F05FC14BF160C1E3
:100290004CF161C14DF162C14EF163C14FF164C1D6
:1002A00050F165C151F166C152F167C153F168C1A6
:1002B00054F166EC01F045C041F146C042F147C03F
:1002C00043F148C044F149C045F11200536AFCECC7
:1002D0002EF073EC30F04BC14AF04CC14BF04DC1E5
:1002E0004CF04EC14DF04FC14EF089EC30F050C192
:1002F0004AF051C14BF052C14CF053C14DF054C1C2
:100300004EF04CEC31F0CFEC00F04CEC31F0120040
:10031000536A090E78EC0AF03AC145F03BC146F049
:100320003CC147F03DC148F03EC149F002EC37F016
:10033000030E4F6E010E506E5284E6EC35F0120043
:10034000536A4A0E78EC0AF046C145F047C146F0C0
:1003500048C147F049C148F04AC149F002EC37F0C2
:10036000030E4F6E010E506EE6EC35F012009DC08C
:1003700045F09EC046F09FC047F0A0C048F0A1C025
:1003800049F002EC37F0040E4F6E020E506EE6ECB0
:1003900035F01200536A000EF86E570EF76EF80E25
:1003A000F66E8AEC0AF0E3DF7AEC0AF079C145F0E8
:1003B0007AC146F07BC147F07CC148F07DC149F06D
:1003C00002EC37F0040E4F6E020E506EE6EC35F084
:1003D00012006EEC0AF015AC11D0000EF86E580E3B
:1003E000F76E540EF66E8AEC0AF0000EF86E580E98
:1003F000F76E660EF66E8AEC0AF070D0000E78EC9E
:100400000AF024EC18F019E2530EE7EC09F0AFDF24
:100410007AEC0AF03AC14BF23BC14CF23CC14DF2CE
:100420003DC14EF23EC14FF25EEC38F0D3EC38F0F5
:1004300050EC3BF07AEC0AF036D087EC2CF07CC024
:1004400030F0E9EC36F0010E4F6E506ABAEC35F040
:10045000410EE7EC09F087EC2CF036C130F037C1E3
:1004600031F0E9EC36F0040E4F6E020E506EBAEC2D
:1004700035F0630E15AE4D0EE7EC09F07AEC0AF09C
:100480003AC145F03BC146F03CC147F03DC148F0A0
:100490003EC149F002EC37F0030E4F6E010E506E74
:1004A0005284E6EC35F0400E78EC0AF0FAEC02F0FB
:1004B0007AEC0AF0A2C030F0A3C031F0CEEC2EF0FE
:1004C00073EC30F05BEC33F002EC37F0030E4F6E60
:1004D000010E506EE6EC35F04FEC04F01200000E09
:1004E00078EC0AF079EC2CF036C130F037C131F0FD
:1004F000FCEC2EF073EC30F05BEC33F002EC37F0F8
:10050000040E4F6E020E506EA3EC36F0E6EC35F0A2
:100510004D0EE7EF09F0400E78EC0AF079EC2CF084
:100520004C0EE7EC09F079EC2CF063C030F0E9EC0C
:1005300036F0030E4F6EE6EC35F0430EE7EC09F0B3
:1005400079EC2CF064C030F065C031F0E9EC36F0A5
:10055000040E4F6EE6EC35F01200000EF86E580EE9
:10056000F76E100EF66E8AEC0AF06FC145F070C19E
:1005700046F071C147F072C148F073C149F002EC16
:1005800037F0050E4F6E030E506EA3EC36F0E6EC1E
:1005900035F0000EF86E580EF76E1A0EF66E8DECF2
:1005A0000AF01200000EF86E580EF76E140EF66E7A
:1005B0008AEC0AF074C145F075C146F076C147F087
:1005C00077C148F078C149F002EC37F0050E4F6E64
:1005D000010E506EA3EC36F0E6EC35F0000EF86E2E
:1005E000580EF76E1E0EF66E8DEC0AF01200400EDD
:1005F00078EC0AF04C0EE7EC09F079EC2CF063C0D3
:1006000030F0E9EC36F0030E4F6EE6EC35F0430EB9
:10061000E7EC09F079EC2CF064C030F065C031F003
:10062000E9EC36F0040E4F6EE6EC35F012008B95D7
:10063000F2D886EC09F011D886EC09F086D886EC61
:1006400009F012008B85E7D886EC09F006D886EC15
:1006500009F07BD886EC09F0120070EC0AF0AFD8F4
:1006600050C145F051C146F052C147F053C148F066
:1006700054C149F04BC14AF04CC14BF04DC14CF054
:100680004EC14DF04FC14EF009EC31F0497E19ECEE
:100690002EF026C069F127C06AF128C06BF150C165
:1006A00045F051C146F052C147F053C148F054C122
:1006B00049F01E0E306ED7EC2EF07EEC30F04CEC94
:1006C00031F04BC14AF04CC14BF04DC14CF04EC122
:1006D0004DF04FC14EF009EC31F0497E19EC2EF08F
:1006E00026C06CF127C06DF128C06EF1000EF86EC7
:1006F000570EF76E920EF66E8AEC0AF087EC2CF02D
:1007000069C130F06AC131F06BC132F0E9EC36F00A
:10071000050E4F6E506ABAEC35F0000EF86E570EAB
:10072000F76E9C0EF66E8AEC0AF087EC2CF06CC12A
:1007300030F06DC131F06EC132F0E9EC36F0050EEB
:100740004F6E506ABAEC35F0120039D8000EF86ED0
:10075000570EF76EA60EF66E8AEC0AF04FC1E8FF50
:1007600081EC0AF04EC1E8FF81EC0AF04DC1E8FFD0
:1007700081EC0AF04CC1E8FF81EC0AF04BC1E8FFC4
:1007800081EC0AF0000EF86E570EF76EAC0EF66EA6
:100790008AEC0AF054C1E8FF81EC0AF053C1E8FF8B
:1007A00081EC0AF052C1E8FF81EC0AF051C1E8FF88
:1007B00081EC0AF050C1E8FF81EC0AF012008BB521
:1007C00015D055C14BF156C14CF157C14DF158C12F
:1007D0004EF159C14FF15AC150F15BC151F15CC1A9
:1007E00052F15DC153F15EC154F114D05FC14BF1C0
:1007F00060C14CF161C14DF162C14EF163C14FF175
:1008000064C150F165C151F166C152F167C153F144
:1008100068C154F1120070EC0AF0D1DF000EF86EDE
:10082000570EF76EA60EF66E8AEC0AF04BC145F035
:100830004CC146F04DC147F04EC148F04FC149F0A0
:100840004CEC37F0070E4F6E060E506E75EC37F01D
:10085000000EF86E570EF76EAC0EF66E8AEC0AF0CC
:1008600050C145F051C146F052C147F053C148F064
:1008700054C149F04CEC37F0070E4F6E060E506E27
:1008800075EC37F0120079EC2CF09AC030F09BC078
:1008900031F09CC032F0E9EC36F0E6EF35F0625210
:1008A00010E1000EF86E540EF76E800EF66E8AECB4
:1008B0000AF0000EF86E540EF76E840EF66E8AEC97
:1008C0000AF0010E626210D0000EF86E540EF76E40
:1008D000880EF66E8AEC0AF0000EF86E540EF76E73
:1008E0008C0EF66E8AEC0AF0020E626210D0000ED8
:1008F000F86E540EF76E900EF66E8AEC0AF0000E4B
:10090000F86E540EF76E940EF66E8AEC0AF0030E33
:10091000626210D0000EF86E540EF76E980EF66EEE
:100920008AEC0AF0000EF86E540EF76E9C0EF66E0E
:100930008AEC0AF0040E626210D0000EF86E540EBB
:10094000F76EA00EF66E8AEC0AF0000EF86E540EEA
:10095000F76EA40EF66E8AEC0AF0050E626210D0F5
:10096000000EF86E540EF76EA80EF66E8AEC0AF0C2
:10097000000EF86E540EF76EAC0EF66E8AEC0AF0AE
:1009800012009BEC0AF0D0B622D004001F2A70ECB3
:100990000AF0000EF86E540EF76E100EF66E8AEC2A
:1009A0000AF0000EF86E540EF76E260EF66E8AEC04
:1009B0000AF087EC2CF01FC030F0E9EC36F0BAEC0E
:1009C00035F089EC09F070EC0AF0148456D0D8ECBC
:1009D0000AF0626AF1EC08F08B88AAEC09F01FECCF
:1009E00011F0C6EC0BF014921E0E1D6E040E1E6E5E
:1009F000000E7A6E33EC11F06BEC11F07DEC11F01F
:100A00008FEC11F059EC11F047EC11F0DAEC00F03A
:100A10000101346B356B366B376B386B396B00010A
:100A200070EC0AF0000EF86E550EF76E1C0EF66EA6
:100A30008AEC0AF070EC0AF0000EF86E550EF76EB4
:100A4000240EF66E8AEC0AF079EC2CF07CC030F0C3
:100A5000E9EC36F0010E4F6EE6EC35F0F5EC08F0FF
:100A600070EC0AF04FEC04F08BEC02F01498BA6BC7
:100A7000BB6BBC6BB56B15841484040044EC09F0AB
:100A8000D8A01CD055EC09F0010E1B6203D067EC16
:100A90001DF012D0020E1B6203D068EC1DF00CD0CA
:100AA0000B0E1B6203D06AEC1DF006D00C0E1B620D
:100AB00003D06DEC1DF000D01B6A14841D2E02D0F3
:100AC0001F0E1D6E1E0E1D6208D014A606D0D6EC99
:100AD00008F0140E8D6F149613801D0E1D6223D026
:100AE00013A021D08D671FD036C130F037C131F04F
:100AF00034C135F035C136F03650315C02E1355045
:100B0000305CD8B410D034C136F135C137F134C1BE
:100B100038F135C139F154EC0EF0F5EC08F08C6B7E
:100B2000A1EC06F014841C0E1D6205D014A403D0A1
:100B30001494E9EC01F01B0E1D620DD07D507C5C1D
:100B4000D8B409D054EC0EF0F5EC08F08C6BA1ECA5
:100B500006F07CC07DF01A0E1D6200D0190E1D62D9
:100B600043D0916741D014AC02D0149C148424EC7F
:100B700018F03AE2158815BE37D0D8EC25F033E3EB
:100B8000640E916F148C148436C130F037C131F08B
:100B900038C135F039C136F03650315C02E135509C
:100BA000305CD8B41CD0D7EC11F010EC01F03FEC65
:100BB00001F023EC00F0230E306E080E316EA2C05F
:100BC00035F0A3C036F03150365C02E13050355C70
:100BD000D8B009D054EC0EF00A0E8E6F148A36C1CC
:100BE00038F137C139F11492180E1D6202D010ECA1
:100BF00001F0170E1D6202D03FEC01F0160E1D62CF
:100C000002D023EC00F0150E1D6208D014B806D0F7
:100C1000D8EC0BF003E32CEC07F0FAD7140E1D62AE
:100C20001FD098EC00F0A4EC32F09DC045F09EC0BF
:100C300046F09FC047F0A0C048F0A1C049F0E7ECE3
:100C400033F00EE29DC079F19EC07AF19FC07BF136
:100C5000A0C07CF1A1C07DF1A4C07EF1A5C07FF150
:100C6000130E1D6224D01E2E02D0040E1E6E010E25
:100C70001E6209D015BC07D040C130F030BE88ECF0
:100C800001F0A0EC01F0020E1E6206D015A404D003
:100C90008C6BA1EC06F01594030E1E6208D08C67D5
:100CA00006D015A804D08C6BA1EC06F01598120E96
:100CB0001D620CD015AA0AD0936708D0926706D09F
:100CC000159AF1EC08F08B98158C1484110E1D62A6
:100CD00012D014AA10D031EC18F00AE28E670BD0B3
:100CE000F5EC08F08C6BA1EC06F0149A148403D098
:100CF0000A0E8E6F00D0100E1D6209D015AC07D001
:100D000015AA05D0F5EC08F0159C14848B880F0EFD
:100D10001D6200D03DEF05F0305092EC06F03150EE
:100D200092EF06F0366E351A3650BFEF0BF0AA0E72
:100D3000BFEC0BF0AA0EBFEC0BF0AA0EBFEF0BF04E
:100D40008C6F8B98356A366AF2DF110E92EC06F0E2
:100D50008C5192EC06F07C5092EC06F062C030F0C0
:100D600063C031F08CEC06F064C030F065C031F047
:100D70008CEC06F036C130F037C131F08CEC06F067
:100D80007EC130F07FC131F08CEC06F03FC130F015
:100D900040C131F08CEC06F0A2C030F0A3C031F0BD
:100DA0008CEC06F08C6707D0730E92EC06F0000E08
:100DB00092EC06F006D0765092EC06F0775092EC6A
:100DC00006F03550BFEC0BF09CEC09F08B8812005C
:100DD0008B98356A366AABDF080E92EC06F00A0E85
:100DE00092EC06F07EC130F07FC131F08CEC06F061
:100DF0003FC130F040C131F08CEC06F0A2C030F0C1
:100E0000A3C031F08CEC06F03550BFEC0BF08B88B2
:100E10001200455092EC06F0465092EC06F0475016
:100E200092EC06F0485092EC06F0495092EF06F032
:100E3000306E8B98356A366A7ADF030E92EC06F0D4
:100E4000140E92EC06F030C0E8FF92EC06F035503C
:100E5000BFEC0BF08B881200B56705D07E0EB36334
:100E60007CD0B52B7AD0010EB56304D0B3C0BAF0F4
:100E7000B52B73D0020EB56357D0B52BB3C0BBF002
:100E8000790EBA6307D0159EBBBF158EBB9FBBC042
:100E9000B6F061D07A0EBA6303D0BBC0B7F05BD0B6
:100EA0007B0EBA6303D0BBC0B8F055D07C0EBA63DA
:100EB00004D0BBC0B9F014864ED0270EBA6303D05D
:100EC000EBEC07F048D0260EBA6303D098EC08F09C
:100ED00042D0250EBA6303D0BBC063F033D0240EDA
:100EE000BA6303D0BBC064F02DD0230EBA6303D025
:100EF000BBC065F027D0220EBA6303D0AEEC07F07A
:100F00002AD01F0EBA630FD070EC0AF079EC2CF0E7
:100F1000BBC0BCF0BB390F0BBB6FBC510F0BBC6F20
:100F2000AFEC1BF018D019D070EC0AF0BA5181EC7C
:100F30000AF0BB5181EC0AF086EC09F070EC0AF083
:100F4000148409D0F5EC08F0148470EC0AF003D096
:100F5000020EB56502D08EEC08F0120015B202D078
:100F600070EC0AF0010EBB6302D01BEF27F0020EFB
:100F7000BB6302D02EEF27F0030EBB6302D041EF1C
:100F800027F0040EBB6302D054EF27F0050EBB63BD
:100F900002D067EF27F0110EBB650DD0550EBB6177
:100FA0000AD0BBC030F030380F0B356EBB510F0B81
:100FB000306E69EF26F0600EBB650CD0BB510F0B95
:100FC000306E305207E0060E306004E030C07CF036
:100FD00027EC11F0120015B202D070EC0AF0BB67DA
:100FE0000CD070EC0AF0000EF86E560EF76EA00EE4
:100FF000F66E8AEC0AF046EC18F0010EBB630CD0DA
:1010000070EC0AF0000EF86E560EF76EA80EF66E33
:101010008AEC0AF044EC18F0020EBB630CD070ECC2
:101020000AF0000EF86E560EF76EB40EF66E8AECED
:101030000AF0A4EC1CF0030EBB630CD070EC0AF0B9
:10104000000EF86E560EF76EDA0EF66E8AEC0AF0A7
:10105000A2EC1CF0040EBB630CD070EC0AF0000E86
:10106000F86E560EF76EBE0EF66E8AEC0AF02CEC99
:101070001CF0050EBB630CD070EC0AF0000EF86E8D
:10108000560EF76ECC0EF66E8AEC0AF067EC1CF08A
:10109000060EBB630CD070EC0AF0000EF86E560E14
:1010A000F76EEA0EF66E8AEC0AF09BEC1BF0070E68
:1010B000BB6302D070EC0AF0080EBB6309D0158246
:1010C0008C6BA1EC06F0600E926FEA0E936F158A9E
:1010D000090EBB630CD070EC0AF0000EF86E560ED1
:1010E000F76EFC0EF66E8AEC0AF0E3EC1BF00A0ECB
:1010F000BB6300D00A0EBB6510D070EC0AF0000E86
:10110000F86E570EF76E080EF66E8AEC0AF00B0EAC
:10111000BB5FBBC0BCF0AFEC1BF000D0BA6BBB6BCD
:10112000BC6BB56B148415B202D070EC0AF01200DF
:10113000BB6702D0626A1DD0010EBB6303D0010EF3
:10114000626E17D0020EBB6303D0020E626E11D026
:10115000030EBB6303D0030E626E0BD0040EBB63A1
:1011600003D0040E626E05D0050EBB6302D0050EDF
:10117000626EF5EC08F0148470EC0AF0000EF86E64
:10118000570EF76ED60EF66E8AEC0AF070EC0AF087
:10119000000EF86E570EF76EE80EF66E8AEC0AF047
:1011A00062503009E7EC09F06250B8D7B65302E15B
:1011B000B75316E087EC2CF0B8C030F0B7C031F070
:1011C000B6C032F0D9EC2FF081EC2DF08EEC2CF083
:1011D0000A0E356EEFEC34F026C034F127C035F13D
:1011E00012005F6A606A616A2AD05F6A63C061F058
:1011F00064C060F065C05FF0626601D020D0010E6F
:10120000626202D05F8E1BD0020E626202D05F8AE1
:1012100016D0030E626204D05F885F8A5F8E0FD0A3
:10122000040E626204D05F8A5F8C5F8E08D0050E68
:10123000626205D05F885F8A5F8C5F8E00D0180E77
:10124000126E5F3260326132D8B08D82D8A08D923A
:1012500040EC09F08D8040EC09F08D9040EC09F0F5
:10126000122EEFD78D843DEC09F08D9496EC09F0A9
:10127000120000000000000000000000000000005C
:101280000000000000001200040081B401D005D06D
:1012900081B601D002D0D8901200D8801200F4DFBD
:1012A000FEE31200F1DFFEE21200F9DF1B6A96ECAA
:1012B00009F081B403D0010E1B6E05D081B603D0B6
:1012C000020E1B6E00D00A0E0E6E8DEC09F044EC7F
:1012D00009F016E30E2EF9D70A0E1B2670EC0AF061
:1012E000000EF86E540EF76E6E0EF66E8AEC0AF073
:1012F0000B0E1B6200D052EC09F070EC0AF0148463
:10130000120044EC09F001E31482120001D801D864
:1013100000D800D800D802D800D800D8320E0DD09E
:10132000280E0BD01E0E09D0140E07D00A0E05D0C1
:10133000050E03D0020E01D0010E04001A6EFA0E43
:10134000186E060E196E182EFED7192EFCD71A2EFF
:10135000F6D71200839E839A839CE0DF300E91D8EB
:10136000EBDF300E8ED8E8DF300E8BD8E5DF200EB5
:1013700088D8DCDF290E78D8080E76D8060E74D807
:10138000010E72D8020E70D80C0E6ED83ED802D85C
:1013900070EF0AF0A5D8000EF86E580EF76E780EB2
:1013A000F66E8AEC0AF0000EF86E580EF76E8A0E92
:1013B000F66E8AEC0AF089EC09F0000EF86E580E11
:1013C000F76E9C0EF66E8AEC0AF089EF09F0206E3B
:1013D00066D82050838A62D8839C60D8839E5ED86A
:1013E000F00B4FD82038F00B4CD0206E2046204612
:1013F000204655D82050400937D8080E0E6E0900F7
:10140000F550E5DF0E2EFBD71200000EF86E140E1D
:10141000F76E280EF66E080E0F6E106A1050E5DF9C
:10142000102A0F2EFBD7120000000000000001154B
:101430000000101010000115000014141400011514
:101440000000151515000115000000000000000047
:1014500000000000000000000000001F040404045D
:101460000000001C04040404206E19D82050F00B66
:10147000839A14D8839C12D8839E10D802D820381F
:10148000F00B040081B0010981B2020981B40409A2
:1014900081B60809816E838E01D8839E12000400F4
:1014A000818EFCDF938EFADF839AF8DF838CF6DF80
:1014B000F5DF5296F3DF838EF1DF81AE5286EEDFE9
:1014C000839EECDF838EEADF839EE8DF52A6F0D7AF
:1014D000939E839CE3DF12000E0EC6D70C0EC4D77A
:1014E000010EC2D7020EC0D7800EBED7C00EBCD729
:1014F0008009BAD7200E6BD70E6EFCDF0E2EFDD7FB
:101500001200216E21380EEC00F061DF21500EEC4C
:1015100000F05DD70900F550EBDF0900F55002E05F
:1015200056DFFBD712000900F5500900F55002E024
:1015300026D9FBD712000F01806A896A1F0E926EAE
:10154000816A8A6A0F0E936E826A8B6AC00E946EED
:10155000836A8C6A000E956E846A8D6A000E966EA0
:101560003F0E896E0F0E8A6E000E8B6E000E8C6E13
:10157000000E8D6E0B0EC16EBF0EC06E000ED06ED3
:10158000D00EF26E000EF16E000EF06E030E9D6E28
:10159000000EA06EA70ED56EA10ECD6E530ECA6EB4
:1015A000340EB16E000EBD6E000EBA6E0001120058
:1015B0000E6A00EE00F0EE6A0E2EFDD7040E0F6EDE
:1015C00001EE00F0EE6A0E2EFDD70F2EFBD71200B3
:1015D0001D0E0DD0190E0BD0150E09D0110E07D00F
:1015E0000D0E05D0090E03D0050E01D0010EC26EFE
:1015F000C282C2B2FED7C4CF95F0C3CF94F012001E
:10160000A6B2FED705C0A9FF06C0A8FFA69EA69C4D
:10161000A684F29EF2BEFDD7550EA76EAA0EA76E47
:10162000A68214A0F28EA6941200A6B2FED705C020
:10163000A9FFA69EA69CA680A8CF06F012000400D3
:10164000DECF06F0DDDF052A0E2EF9D708D0040024
:10165000ECDF06C0DEFF052A0E2EF9D7120070EC73
:101660000AF0000EF86E580EF76E300EF66E8AEC29
:101670000AF0000EF86E580EF76E420EF66E8AEC07
:101680000AF089EC09F0148470EF0AF004008394E6
:1016900065EC0BF021D81ED8838409D820D0040033
:1016A000838465EC0BF018D815D8839402D8839600
:1016B00002D006D00AD000000000000000000000A8
:1016C000000000000000000000000000000000001A
:1016D000000012008386ECD795949596F6D79584F2
:1016E0009586F3D7DCDFA00E0BD807BEFBD70950D9
:1016F00007D807BEF7D7085003D807BEF3D71200A4
:10170000839665EC0BF00C6EE7DF080E0D6E04009F
:10171000838465EC0BF00CAE8394CBDFDBDFC7DF9B
:101720000C360D2EF4D7958465EC0BF0959665EC90
:101730000BF0079ECFDF83B4078EBBDF839665EC8B
:101740000BF01200080E0D6E0A6A04000A360A90A9
:10175000EADF07BE0A800D2EF8D71200C3DF0B5058
:10176000CFDF94D793DFBEDF9ADFA10EC9DF07BEBC
:10177000F9D7E8DF8BD79EAAFED7AE501200ACA2F5
:10178000FED79EA8FCD7AD6E9CEF09F005EE00F0E9
:10179000EACFB0F0E9CFAFF0EACFB2F0E9CFB1F0E5
:1017A0001D0EAF6EAC94AC8AAB889D8AAB8E1200D6
:1017B000B1C0E1FFB2C0E2FFAF51E15C02E1D890FD
:1017C0001200E650B36FF10EE15C02E115EE00F09D
:1017D000E1CFB1F0E2CFB2F0B351D8801200216E68
:1017E00021380EEC00F0BFEC0BF021500EEC00F0B5
:1017F000BFEF0BF0200EBFEF0BF00D0EBFEF0BF0A5
:101800000AEC0CF0566604D0556602D0D89012004F
:10181000D8801200D76AD66A1580CD9079EC2CF06A
:10182000D30E316E000E306E5AC035F035AE04D096
:1018300036683768386839680CEC30F03150CF6E54
:101840003050CE6ECD80928A15B0FED7576A586A56
:10185000596AD650586ED750596E898A899A570658
:1018600006E0D650585C898AF9E0929A03D0556A0E
:10187000566A12D057C030F058C031F059C032F01B
:10188000E7EC2EF073EC30F05BEC33F019EC2EF05B
:1018900026C055F027C056F0120070EC0AF079EC23
:1018A0002CF057C030F058C031F059C032F0E9EC9C
:1018B00036F0060E4F6E040E506EBAEC35F0000E88
:1018C000F86E540EF76EC40EF66E8DEC0AF0400EF4
:1018D00078EC0AF087EC2CF055C030F056C031F0AF
:1018E000E9EC36F0040E4F6E020E506EBAEC35F095
:1018F000000EF86E540EF76EC40EF66E8DEC0AF004
:1019000089EC09F070EC0AF014841200B3EC0BF0CF
:101910000AC030F0082AD8B4092AB3EC0BF00AC088
:1019200031F0082AD8B4092AB3EC0BF00AC032F01F
:10193000082AD8B4092AB3EC0BF00AC033F0E868DF
:10194000305C08E030C062F031C063F032C064F057
:1019500033C065F0120062C00BF0AEEC0BF0082A49
:10196000D8B4092A63C00BF0AEEC0BF0082AD8B447
:10197000092A64C00BF0AEEC0BF0082AD8B4092A8F
:1019800065C00BF0AEEC0BF0120079EC2CF036C118
:1019900030F037C131F0306604D0316602D0D880E3
:1019A00043D0960E356EFAEC2FF081EC2DF08EECD4
:1019B0002CF0040E356E7BEC34F0010E7C6205D009
:1019C000000E306E000E316E26D0020E7C6205D005
:1019D000880E306E2C0E316E1ED0030E7C6205D048
:1019E000100E306E590E316E16D0040E7C6205D08A
:1019F000980E306E850E316E0ED0050E7C6205D0CD
:101A0000200E306EB20E316E06D087EC2CF0010E37
:101A10007C6E7CC07DF0305026263150272226C0B7
:101A200008F027C009F0D890120036C18EF137C1F6
:101A30008FF136C130F037C131F0306603D03166F6
:101A400001D0E4D070EC0AF0000EF86E550EF76E7F
:101A5000300EF66E8AEC0AF089EC09F0C80E806F41
:101A6000000E816F3150815D02E13050805DD8A061
:101A700005D0B40E7E6E000E7F6EA2D0860E806FF3
:101A8000010E816F3150815D02E13050805DD8A040
:101A900005D0540E7E6E010E7F6E92D01C0E806FAC
:101AA000020E816F3150815D02E13050805DD8A01F
:101AB00005D0120E7E6E020E7F6E82D0DA0E806F1F
:101AC000020E816F3150815D02E13050805DD8A0FF
:101AD00005D0B20E7E6E020E7F6E72D0FC0E806F4D
:101AE000030E816F3150815D02E13050805DD8A0DE
:101AF00005D0E80E7E6E030E7F6E62D0A00E806F62
:101B0000050E816F3150815D02E13050805DD8A0BB
:101B100005D06E0E7E6E050E7F6E52D01C0E806F4D
:101B2000070E816F3150815D02E13050805DD8A099
:101B300005D0080E7E6E070E7F6E42D0700E806F4D
:101B4000080E816F3150815D02E13050805DD8A078
:101B500005D02A0E7E6E080E7F6E32D0280E806F62
:101B60000A0E816F3150815D02E13050805DD8A056
:101B700005D00A0E7E6E0A0E7F6E22D0A40E806FF4
:101B80000B0E816F3150815D02E13050805DD8A035
:101B900005D0E60E7E6E0A0E7F6E12D07EC030F04B
:101BA0007FC031F030660CD031660AD02FD080C0B3
:101BB00030F081C031F0306603D0316601D026D0DC
:101BC0007EC036F17FC037F1C5EC0CF00CE2ABEC17
:101BD0000CF07E2AD8B47F2A7F50815D02E17E50CE
:101BE000805DD8B0EDD770EC0AF0000EF86E550E9F
:101BF000F76E0A0EF66E8AEC0AF0050EA0EC06F0FF
:101C000089EC09F070EC0AF0D89018D0000EF86E4C
:101C1000570EF76E3C0EF66E8AEC0AF0000EF86E68
:101C2000570EF76E4E0EF66E8AEC0AF0060EA0EC1A
:101C300006F089EC09F070EC0AF0D8808EC136F11C
:101C40008FC137F11200C5EC0CF015E270EC0AF010
:101C5000ABEC0CF0000EF86E550EF76E0A0EF66E39
:101C60008AEC0AF0050EA0EC06F089EC09F070ECA5
:101C70000AF0D8901200000EF86E570EF76E3C0E68
:101C8000F66E8AEC0AF0000EF86E570EF76E4E0EE6
:101C9000F66E8AEC0AF0060EA0EC06F089EC09F06C
:101CA00070EC0AF0D8801200C5EC0CF002E286EC71
:101CB0000CF01200536AD7EC2EF073EC30F08BB5B9
:101CC0000BD05AC14AF05BC14BF05CC14CF05DC116
:101CD0004DF05EC14EF00AD064C14AF065C14BF0D0
:101CE00066C14CF067C14DF068C14EF046EC31F072
:101CF0008BB50BD055C14AF056C14BF057C14CF0D3
:101D000058C14DF059C14EF00AD05FC14AF060C1D0
:101D10004BF061C14CF062C14DF063C14EF009EC73
:101D200031F019EC2EF0120070EC0AF0666A6EECDD
:101D30000AF0000EF86E540EF76E460EF66E8AEC40
:101D40000AF087EC2CF069C130F06AC131F0E9EC9F
:101D500036F0050E4F6E506ABAEC35F0000EF86E94
:101D6000540EF76E520EF66E8AEC0AF087EC2CF0E9
:101D70006CC130F06DC131F0E9EC36F0050E4F6EFC
:101D8000506ABAEC35F07AEC0FF0795208E079AE8F
:101D9000E4EC0EF079BE2CEC0FF0796AC8D744EC75
:101DA00009F0F3E355EC09F0020E1B6203D06EEC70
:101DB0000AF009D0010E1B6206D0662A060E666282
:101DC00001D0666AB4D7120069C130F06AC131F03F
:101DD0006CC135F06DC136F0666603D0302AD8B4D8
:101DE000312A010E666208D00A0E326E000E336E82
:101DF0003250302633503122020E666208D0640E13
:101E0000326E000E336E3250302633503122030EC4
:101E1000666203D0352AD8B4362A040E666208D02A
:101E20000A0E326E000E336E325035263350362293
:101E3000050E666208D0640E326E000E336E3250AC
:101E400035263350362230C069F131C06AF135C0D1
:101E50006CF136C06DF1120069C130F06AC131F029
:101E60006CC135F06DC136F0666606D0300630289C
:101E7000D8B43106D8B43052010E666208D00A0ECA
:101E8000326E000E336E3250305E3350315A020ED5
:101E9000666208D0640E326E000E336E3250305ED1
:101EA0003350315A030E666206D035063528D8B451
:101EB0003606D8B43552040E666208D00A0E326E69
:101EC000000E336E3250355E3350365A050E666260
:101ED00008D0640E326E000E336E3250355E3350D1
:101EE000365A30C069F131C06AF135C06CF136C084
:101EF0006DF11200666602D00E0E18D0010E6662F9
:101F000002D00D0E13D0020E666202D00C0E0ED05F
:101F1000030E666202D04E0E09D0040E666202D035
:101F20004D0E04D0050E666201D04C0E78EC0AF01E
:101F30006CEC0AF012008B95306A5AEC0EF026C059
:101F400069F127C06AF1E20E306E5AEC0EF026C03D
:101F50006CF127C06DF194EC0EF06AEF10F08B85F8
:101F6000306A5AEC0EF026C069F127C06AF1E20E21
:101F7000306E5AEC0EF026C06CF127C06DF194EC77
:101F80000EF06AEF10F0D8909A379B379C37D890B4
:101F90009A379B379C3787EC2CF08BB505D096C0D1
:101FA00030F097C031F004D098C030F099C031F0D3
:101FB00030509A2731509B2332509C2379EC2CF0DF
:101FC0009AC030F09BC031F09CC032F0050E356EE7
:101FD000EFEC34F026C09AF027C09BF028C09CF0AC
:101FE00012008B8501D08B959A6B9B6B9C6B70EC70
:101FF0000AF08BB509D0000EF86E570EF76E600E22
:10200000F66E8AEC0AF008D0000EF86E570EF76EE6
:10201000720EF66E8AEC0AF0000EF86E570EF76E2E
:10202000840EF66E8AEC0AF0000EF86E570EF76E0C
:10203000880EF66E8AEC0AF08CEC09F0C2EC11F016
:10204000C3EC0FF043EC04F044EC09F0D2E355ECA0
:1020500009F0020E1B6209D0EEEC27F09AC069F17C
:102060009BC06AF19CC06BF106D0010E1B6202D0CE
:1020700005EF11F0BED7000EF86E570EF76E840E06
:10208000F66E8AEC0AF0000EF86E570EF76E9C0E94
:10209000F66E8AEC0AF08CEC09F0C2EC11F0C3EC9D
:1020A0000FF043EC04F044EC09F0E5E355EC09F0E3
:1020B000020E1B6209D0EEEC27F09AC06CF19BC0B7
:1020C0006DF19CC06EF106D0010E1B6202D005EFCF
:1020D00011F0D1D779EC2CF069C130F06AC131F040
:1020E0006BC132F0FCEC2EF073EC30F0C6EC2CF04F
:1020F00079EC2CF06CC130F06DC131F06EC132F072
:10210000FCEC2EF073EC30F04AEC2DF0A5EC2CF04A
:10211000DCEC2CF046EC31F0BBEC2CF0410E496EBF
:10212000F00E486E456A466A476A09EC31F045C0D0
:102130004BF146C04CF147C04DF148C04EF149C08B
:102140004FF10EC24AF00FC24BF010C24CF011C258
:102150004DF012C24EF089EC30F0497E45C050F18E
:1021600046C051F147C052F148C053F149C054F143
:1021700070EC0AF00EEC04F086EC09F0000EF86E3C
:10218000570EF76EB20EF66E8AEC0AF0000EF86E7D
:10219000570EF76EC40EF66E8AEC0AF04FEC09F09B
:1021A00055EC09F0020E1B6230D08BB517D04BC135
:1021B00055F14CC156F14DC157F14EC158F14FC1C7
:1021C00059F150C15AF151C15BF152C15CF153C197
:1021D0005DF154C15EF161EC11F021D04BC15FF1B2
:1021E0004CC160F14DC161F14EC162F14FC163F16B
:1021F00050C164F151C165F152C166F153C167F13B
:1022000054C168F173EC11F00AD070EC0AF0000EC2
:10221000F86E570EF76E2A0EF66E8AEC0AF089EC0D
:1022200009F070EC0AF08B95120020EE13F0010E0D
:102230000E6E010E056E1FEC0BF08DEF09F020EE17
:1022400013F0010E0E6E010E056E27EF0BF020EE5F
:102250007CF0010E0E6E000E056E1FEC0BF097EC7D
:1022600011F08DEF09F020EE7CF0010E0E6E000EE5
:10227000056E27EC0BF097EF11F020EEAAF0010E9F
:102280000E6E180E056E1FEC0BF08DEF09F020EEB0
:10229000AAF0010E0E6E180E056E27EF0BF020EE61
:1022A000A9F0010E0E6E170E056E1FEC0BF08DEFF0
:1022B00009F020EEA9F0010E0E6E170E056E27EF45
:1022C0000BF021EE55F00A0E0E6E030E056E1FEC9C
:1022D0000BF08DEF09F021EE55F00A0E0E6E030E95
:1022E000056E27EF0BF021EE5FF00A0E0E6E0D0E5D
:1022F000056E1FEC0BF08DEF09F021EE5FF00A0E7A
:102300000E6E0D0E056E27EF0BF020EE5AF0010E4B
:102310000E6E020E056E1FEC0BF08DEF09F020EE35
:102320005AF0010E0E6E020E056E27EF0BF08B9227
:102330008B948B968C908B92010E7C6201D08B8259
:10234000020E7C6201D08B84030E7C6201D08B86EE
:10235000040E7C6201D08C80050E7C6201D08B82E1
:1023600012008A6703D096EC09F00BD0010E8A6345
:1023700003D090EC09F005D0020E8A6302D08DECF8
:1023800009F01200200E0E6E966B976B986B996B8E
:10239000F6EC0AF09451962795519723F4EC0AF045
:1023A00094519827955199230E2EF2D71200D9DF18
:1023B000E9DF96C06FF097C070F0800E306E0C0EA3
:1023C000316E30506F263150702298516F5E9951A6
:1023D000705A70AE04D0640E6F6E000E706E1200F4
:1023E00063C073F064C074F065C075F096C08AF184
:1023F00097C08BF198C08CF199C08DF112008B6B56
:1024000015B68B8D70EC0AF06F6A706A636A646A45
:10241000656AF5EC08F096EC09F0D7EC11F06FC0A6
:1024200071F070C072F063C073F064C074F065C086
:1024300075F0F9EC12F08A6BF5EC08F0D7EC11F0BE
:102440007050725C02E16F50715CD8B006D06FC002
:1024500071F070C072F0F0EC11F01ED9EDE32CECCD
:1024600013F01AEC18F003E314828B8742D073C088
:1024700063F074C064F075C065F0F5EC08F0F9EC39
:1024800012F08BBD11D0E00E306E020E316EA2C084
:1024900035F0A3C036F03150365C02E13050355C87
:1024A000D8B002D08B8B25D071EC15F050EC17F022
:1024B00008EC15F01AEC18F003E314828B8719D09E
:1024C0008BB117D0010E776201D007D05AEC15F00E
:1024D000FEEC15F050EC17F0EBD773C063F074C04E
:1024E00064F075C065F0F5EC08F096EC09F0F9ECD5
:1024F00012F012008B6B15B68B8D70EC0AF06F6AC0
:10250000706A636A646A656AF5EC08F096EC09F033
:10251000D7EC11F06FC071F070C072F063C073F04F
:1025200064C074F065C075F0F9EC12F08A6B636AF0
:10253000F5EC08F0D7EC11F07050725C02E16F50CE
:10254000715CD8B006D06FC071F070C072F0F0EC62
:1025500011F0B9D8EDE32CEC13F01AEC18F003E30A
:1025600014828B8742D073C063F074C064F075C06E
:1025700065F0F5EC08F0F9EC12F08BBD11D0E00E2F
:10258000306E020E316EA2C035F0A3C036F031506D
:10259000365C02E13050355CD8B002D08B8B25D050
:1025A00063EC15F028EC17F0CBEC14F01AEC18F0F3
:1025B00003E314828B8719D08BB117D0010E76629A
:1025C00001D007D053EC15F0F8EC15F028EC17F01B
:1025D000EBD773C063F074C064F075C065F0F5ECC0
:1025E00008F096EC09F0F9EC12F01200D7EC11F0BB
:1025F00006D0D7EC11F08BEC02F04FEC04F010ECAD
:1026000001F03AC185F13BC186F13CC187F13DC182
:1026100088F13EC189F13FEC01F023EC00F098EC29
:1026200000F09DC080F19EC081F19FC082F1A0C0EA
:1026300083F1A1C084F19DC079F19EC07AF19FC061
:102640007BF1A0C07CF1A1C07DF1A4C07EF1A5C04A
:102650007FF1E9EC01F0120063C098F164C099F1D8
:1026600065C09AF173C063F074C064F075C065F022
:102670008AC196F08BC197F08CC198F08DC199F00A
:102680008BEC02F04FEC04F0B6DF98C163F099C117
:1026900064F09AC165F01200656608D0646606D0E1
:1026A000080E646E000E656ED8900BD0D89064361C
:1026B000653665A606D0FF0E646E070E656ED8807F
:1026C00001D0D8901200636603D0632AD89000D05E
:1026D000D8906336D8A002D06368D88012008B6B84
:1026E00015B602D08B8D8B8370EC0AF06F6A706A1E
:1026F000F5EC08F096EC09F0D7EC11F06FC071F032
:1027000070C072F063C073F064C074F065C075F09F
:102710008A6BF9EC12F0626604D091EC15F0D2EFFE
:1027200012F0050E626204D0B8EC15F056EF12F00C
:102730008FEC15F06ED08B6B15B68B8D70EC0AF0AC
:102740006F6A706A636A646A656AF5EC08F096EC11
:1027500009F0D7EC11F06FC071F070C072F063C077
:1027600073F064C074F065C075F0F9EC12F0090EF6
:10277000A0EC06F0626602D07AEF12F0050E6262FB
:1027800002D0FFEF11F08A6B636A646A656AF5EC48
:1027900008F0D7EC11F07050725C02E16F50715C80
:1027A000D8B006D06FC071F070C072F0F0EC11F0CC
:1027B00073DFEDE32CEC13F0090EA0EC06F083DFE1
:1027C000E4E31AEC18F003E314828B8748D073C05B
:1027D00063F074C064F075C065F0F5EC08F0F9ECD6
:1027E00012F0090EA0EC06F08BBD11D0E00E306E99
:1027F000020E316EA2C035F0A3C036F03150365C07
:1028000002E13050355CD8B002D08B8B28D061EC1F
:1028100015F026EC17F030EC14F01AEC18F003E386
:1028200014828B8710D08BB11AD0010E766204D03F
:10283000010E776201D007D051EC15F005EC16F0CF
:1028400026EC17F0E8D773C063F074C064F075C06D
:1028500065F0F5EC08F096EC09F0F9EC12F01200D6
:1028600068C08EF169C08FF168C064F069C065F01E
:102870006CC063F0F5EC08F0F9EC12F00A0EA0EC75
:1028800006F06FC071F070C072F063C073F064C086
:1028900074F065C075F06CC063F08EC168F08FC1D4
:1028A00069F068C064F069C065F0F5EC08F0D7EC39
:1028B00011F07050725C02E16F50715CD8B006D0BC
:1028C0006FC071F070C072F0F0EC11F079EC2CF088
:1028D00068C030F069C031F077C035F00CEC30F0F2
:1028E00030C068F031C069F069506B5C02E168503B
:1028F0006A5CD8B0D6D72CEC13F00A0EA0EC06F028
:1029000079EC2CF06CC030F076C035F00CEC30F087
:1029100030C06CF0366A6DC035F03150365C02E183
:102920003050355CD8B0B7D773C063F074C064F072
:1029300075C065F0F5EC08F096EC09F0F9EC12F0D2
:102940000A0EA0EC06F08BA314D08BA912D0540E63
:10295000306E0A0E316EA2C035F0A3C036F036508C
:10296000315C02E13550305CD8B003D08B9B8B8159
:1029700011D0230E306E080E316EA2C035F0A3C008
:1029800036F03650315C02E13550305CD8B002D0C0
:102990008B9B8B8112006CC063F0646A656AF5ECF6
:1029A00008F0F9EC12F00A0EA0EC06F06FC071F01E
:1029B00070C072F063C073F064C074F065C075F0ED
:1029C0006CC063F0F5EC08F0D7EC11F07050725C5D
:1029D00002E16F50715CD8B006D06FC071F070C06A
:1029E00072F0F0EC11F079EC2CF06CC030F076C0A5
:1029F00035F00CEC30F030C06CF0366A6DC035F05C
:102A00003150365C02E13050355CD8B0D9D78CD724
:102A100068C08EF169C08FF168C064F069C065F06C
:102A2000636AF5EC08F0F9EC12F00A0EA0EC06F07F
:102A30006FC071F070C072F063C073F064C074F066
:102A400065C075F068C064F069C065F0F5EC08F029
:102A5000D7EC11F07050725C02E16F50715CD8B02D
:102A60000AD06FC071F070C072F063C073F064C0C0
:102A700074F065C075F079EC2CF068C030F069C076
:102A800031F077C035F00CEC30F030C068F031C078
:102A900069F069506B5C02E168506A5CD8B0D2D7CB
:102AA00043D701D807D0D8907632766602D0010E8F
:102AB000766E1200D8907732776602D0010E776E6C
:102AC000120001D80ED063C06DF06DBE03D0D89057
:102AD0006D3602D0FF0E6D6E63C06CF0D8906C3214
:102AE000120064C06AF065C06BF06BB404D0D8907B
:102AF0006A366B3604D0FF0E6A6E070E6B6E64C0CA
:102B000068F065C069F0696606D0080E686003D099
:102B1000686A696A03D0D89069326832120001D8B5
:102B200027D079EC2CF063C030F0020E356EEFEC5C
:102B300034F08EEC2CF063C035F00CEC30F0FF0E6E
:102B4000356E000E366E3150365C02E13050355C29
:102B5000D8B002D0306805D0080E306002D0080E20
:102B6000306E30C06DF063C06CF0D8906C321200E3
:102B700079EC2CF064C030F065C031F0020E356E97
:102B8000EFEC34F08EEC2CF064C035F065C036F01C
:102B90000CEC30F0FF0E356E070E366E3150365CA1
:102BA00002E13050355CD8B005D0FF0E306E070E14
:102BB000316E0FD0080E356E000E366E3650315C19
:102BC00002E13550305CD8B004D0080E306E000EF3
:102BD000316E30C06AF031C06BF064C068F065C01F
:102BE00069F0D890693268321200020E6E6E11D010
:102BF000040E6E6E0ED0020E6E6E90D0040E6E6ECF
:102C00008DD0020E6E6E05D889D0040E6E6E01D87E
:102C100085D079EC2CF06EC030F076C035F07BECCE
:102C200034F030C08EF131C08FF132C090F133C03A
:102C300091F134C092F179EC2CF063C030F08EC188
:102C400035F08FC136F090C137F091C138F092C1A4
:102C500039F00CEC30F0FF0E356E000E366E315050
:102C6000365C02E13050355CD8B021D06D6879EC2B
:102C70002CF06DC030F08EC135F08FC136F090C1B0
:102C800037F091C138F092C139F0F7EC2FF08EC1D6
:102C900035F08FC136F090C137F091C138F092C154
:102CA00039F0F7EC2FF030C06CF037D002D030C0E4
:102CB0006DF079EC2CF063C030F08EC135F08FC12F
:102CC00036F090C137F091C138F092C139F0F7EC8D
:102CD0002FF034AE20D06C6A79EC2CF06CC030F060
:102CE0008EC135F08FC136F090C137F091C138F008
:102CF00092C139F00CEC30F08EC135F08FC136F056
:102D000090C137F091C138F092C139F00CEC30F03D
:102D100030C06DF002D030C06CF0120079EC2CF0B5
:102D20006EC030F077C035F07BEC34F030C08EF1FF
:102D300031C08FF132C090F133C091F134C092F1C3
:102D400079EC2CF064C030F065C031F08EC135F004
:102D50008FC136F090C137F091C138F092C139F08F
:102D60000CEC30F0FF0E356E070E366E3150365CCF
:102D700002E13050355CD8B027D0FF0E6A6E070EE6
:102D80006B6E79EC2CF06AC030F06BC031F08EC104
:102D900035F08FC136F090C137F091C138F092C153
:102DA00039F0F7EC2FF08EC135F08FC136F090C1BD
:102DB00037F091C138F092C139F0F7EC2FF030C004
:102DC00068F031C069F041D030C06AF031C06BF0BA
:102DD00079EC2CF064C030F065C031F08EC135F074
:102DE0008FC136F090C137F091C138F092C139F0FF
:102DF000F7EC2FF034AE25D0686A696A79EC2CF0D4
:102E000068C030F069C031F08EC135F08FC136F046
:102E100090C137F091C138F092C139F00CEC30F02C
:102E20008EC135F08FC136F090C137F091C138F0C6
:102E300092C139F00CEC30F030C06AF031C06BF068
:102E400004D030C068F031C069F0120001D828D039
:102E500079EC2CF06DC030F06CC035F0F7EC2FF051
:102E6000400E266403D0100E766E19D0200E266414
:102E700003D0080E766E13D0100E266403D0040E15
:102E8000766E0DD0080E266403D0020E766E07D043
:102E9000040E266402D0010E766E010E766E1200CC
:102EA00079EC2CF06AC030F06BC031F068C035F0BE
:102EB00069C036F0F7EC2FF0000E356E020E366E5C
:102EC0002750365C02E12650355CD8B003D0800E26
:102ED000776E63D0000E356E010E366E2750365C6D
:102EE00002E12650355CD8B003D0400E776E55D045
:102EF000800E356E000E366E2750365C02E126508D
:102F0000355CD8B003D0200E776E47D0400E356EBA
:102F1000000E366E2750365C02E12650355CD8B084
:102F200003D0100E776E39D0200E356E000E366E3F
:102F30002750365C02E12650355CD8B003D0080E2D
:102F4000776E2BD0100E356E000E366E2750365C25
:102F500002E12650355CD8B003D0040E776E1DD048
:102F6000080E356E000E366E2750365C02E1265094
:102F7000355CD8B003D0020E776E0FD0040E356EDC
:102F8000000E366E2750365C02E12650355CD8B014
:102F900002D0010E776E010E776E120070EC0AF00F
:102FA0004C0EE7EC09F087EC2CF06CC030F0E9EC4B
:102FB00036F0050E4F6EBAEC35F087EC2CF06DC094
:102FC00030F0E9EC36F0050E4F6EBAEC35F087ECD8
:102FD0002CF076C030F0E9EC36F0040E4F6EBAEC0F
:102FE00035F0400E78EC0AF0430EE7EC09F087EC80
:102FF0002CF068C030F069C031F0E9EC36F0050E15
:103000004F6EBAEC35F087EC2CF06AC030F06BC034
:1030100031F0E9EC36F0050E4F6EBAEC35F087EC86
:103020002CF077C030F0E9EC36F0040E4F6EBAECBD
:1030300035F01200D8EC11F010EC01F03EC130F088
:10304000D89030BED8801200D8EC11F09751AC5D0A
:1030500002E19651AB5DD8B002D0D89001D0D880B3
:103060001200D8EC11F0AE51975D02E1AD51965DC2
:10307000D8B002D0D89001D0D8801200906703D089
:103080008F6701D014821200158601D0159652EC7C
:1030900009F0F1EC08F01492000EF86E570EF76E7E
:1030A000180EF66E8AEC0AF0010EA0EC06F0B80ECF
:1030B0008F6F0B0E906F3EEC18F014B2CED181ECF6
:1030C00009F014B2CAD124EC18F0F5E2D8EC25F0DE
:1030D000F2E38B9F31EC18F002E38B8FD5D1070E12
:1030E000A0EC06F00101796B7A6B806B816B0001BB
:1030F00070EC0AF0000EF86E540EF76EB00EF66E1D
:103100008AEC0AF06FEC02F089EC09F070EC0AF03E
:10311000716A726A71C000F172C001F171C007F189
:1031200072C008F171C00EF172C00FF171C015F1DB
:1031300072C016F171C01CF172C01DF171C023F193
:1031400072C024F1010E626E9BEC13F073C009F1A2
:1031500074C00AF175C00BF171C007F172C008F1BB
:1031600076C00CF177C00DF114B278D08BBB02D0D1
:103170008BB13ED1030E626E9BEC13F073C017F15E
:1031800074C018F175C019F171C015F172C016F153
:1031900076C01AF177C01BF114B260D08BBB02D09D
:1031A0008BB126D1020E626E9BEC13F073C010F14E
:1031B00074C011F175C012F171C00EF172C00FF13F
:1031C00076C013F177C014F114B248D08BBB02D093
:1031D0008BB10ED1040E626E9BEC13F073C01EF126
:1031E00074C01FF175C020F171C01CF172C01DF1D7
:1031F00076C021F177C022F114B230D08BBB02D05F
:103200008BB1F6D02BD0050E626EFFEC11F073C0BF
:1032100025F174C026F175C027F171C023F172C089
:1032200024F176C028F177C029F114B217D08BB100
:10323000DFD0626A7AEC12F073C002F174C003F15D
:1032400075C004F171C000F172C001F176C005F1E2
:1032500077C006F114B202D08BB1CAD007C130F0EA
:1032600008C131F00EC135F00FC136F03150365C77
:1032700002E13050355CD8B011D009C163F00AC109
:1032800064F00BC165F007C16FF008C170F00CC1AC
:1032900076F00DC177F0010E626E10D010C163F0B0
:1032A00011C164F012C165F00EC16FF00FC170F072
:1032B00013C176F014C177F0020E626E15C130F0C2
:1032C00016C131F03150705C02E130506F5CD8B003
:1032D00010D017C163F018C164F019C165F015C1B1
:1032E0006FF016C170F01AC176F01BC177F0030EB3
:1032F000626E1CC130F01DC131F03150705C02E1D2
:1033000030506F5CD8B010D01EC163F01FC164F0A4
:1033100020C165F01CC16FF01DC170F021C176F0B5
:1033200022C177F0040E626E35D000C130F001C1C9
:1033300031F03150705C02E130506F5CD8B00FD08A
:1033400002C163F003C164F004C165F000C16FF015
:1033500001C170F005C176F006C177F0626A23C141
:1033600030F024C131F03150705C02E130506F5CBC
:10337000D8B010D025C163F026C164F027C165F034
:1033800023C16FF024C170F028C176F029C177F015
:10339000050E626EF5EC08F0F6EC12F0760E306E6B
:1033A000050E316EA2C035F0A3C036F03150365C48
:1033B00002E13050355CD8B01BD08BB74ED070ECEA
:1033C0000AF0000EF86E540EF76EEC0EF66E8AECF4
:1033D0000AF0000EF86E540EF76EC80EF66E8AEC08
:1033E0000AF0030EA0EC06F089EC09F0B2D822D066
:1033F00070EC0AF0000EF86E540EF76EEC0EF66EDE
:103400008AEC0AF0000EF86E550EF76E020EF66E9C
:103410008AEC0AF0F5EC08F0F6EC12F0020EA0ECE3
:1034200006F089EC09F095D8ADEC1BF036C138F107
:1034300037C139F189EC09F070EC0AF055EC1AF05B
:1034400080C18EF181C18FF182C190F183C191F170
:1034500084C192F17AEC1AF01BD070EC0AF0000EE5
:10346000F86E540EF76EEC0EF66E8AEC0AF0000E53
:10347000F86E540EF76EDA0EF66E8AEC0AF0030E52
:10348000A0EC06F089EC09F064D889EC09F000D0D2
:1034900070EC0AF0148414928C6BA1EC06F08C6B27
:1034A000A1EC06F089EC09F01200000EF86E580E3F
:1034B000F76E020EF66E8AEC0AF087EC2CF076C0FE
:1034C00030F0E9EC36F0030E4F6EE6EC35F0000E0E
:1034D000F86E580EF76E0C0EF66E8AEC0AF087EC5A
:1034E0002CF077C030F0E9EC36F0030E4F6EE6ECCE
:1034F00035F01200000EF86E570EF76EFC0EF66EE9
:103500008AEC0AF08EC145F08FC146F090C147F0B9
:1035100091C148F092C149F002EC37F0040E4F6EB1
:10352000020E506EE6EC35F07AEC0AF085C14BF2F3
:1035300086C14CF287C14DF288C14EF289C14FF26B
:103540005EEC38F0D3EC38F050EC3BF088EC09F04E
:1035500012008BAF04D00C0EA0EC06F00BD08BA7A2
:1035600006D00B0EA0EC06F088EC09F003D0040E98
:10357000A0EC06F08B78D8EC11F0400E306E1F0EE8
:10358000316E9751315C02E19651305CD8B003D076
:1035900089EC09F0EFD78B88F5EC08F089EC09F09D
:1035A0001200636A646A656A1200C80E306E000E0B
:1035B000316E5650315C02E15550305CD8A005D0D8
:1035C000040E766E100E776E3FD0900E306E010EA8
:1035D000316E5650315C02E15550305CD8A005D0B8
:1035E000030E766E0A0E776E2FD0200E306E030E0D
:1035F000316E5650315C02E15550305CD8A005D098
:10360000020E766E040E776E1FD0D00E306E070E4F
:10361000316E5650315C02E15550305CD8A005D077
:10362000010E766E020E776E0FD0B80E306E0B0E56
:10363000316E5650315C02E15550305CD8A004D058
:10364000010E766E010E776E1200AFDFC80E306E7F
:10365000000E316E5650315C02E15550305CD8A0FE
:1036600009D0640E636EE80E646E030E656E0A0E7A
:10367000886F50D0900E306E010E316E5650315C16
:1036800002E15550305CD8A009D0500E636EF40EA4
:10369000646E010E656E0A0E886F3CD0200E306E8F
:1036A000030E316E5650315C02E15550305CD8A0AB
:1036B00009D0140E636E640E646E000E656E080E03
:1036C000886F28D0D00E306E070E316E5650315CA8
:1036D00002E15550305CD8A009D00A0E636E320E5C
:1036E000646E000E656E060E886F14D0B80E306ED4
:1036F0000B0E316E5650315C02E15550305CD8A053
:1037000009D0050E636E050E646E000E656E0A0E1E
:10371000886F00D0626604D0060E786E636A0AD0A5
:10372000050E626205D0040E786E646A656A02D086
:10373000050E786E120079EC2CF079C18EF17AC109
:103740008FF17BC190F17CC191F17DC192F1E8ECE8
:1037500006F07AEC1AF048EF1AF0BB6BBC6B36C17E
:103760008EF137C18FF136C17EF037C17FF036C19F
:1037700080F037C181F087EC2CF0BBC030F03050C6
:103780007E5E31507F5A87EC2CF0BCC030F0305058
:10379000802731508123CEEC0DF08EC136F18FC1E0
:1037A00037F1BB6BBC6B48EF1AF070EC0AF0000EFF
:1037B000F86E570EF76E140EF66E8AEC0AF089EC6E
:1037C00009F070EC0AF015EC0DF048EF1AF052EC2D
:1037D00009F063C02CF164C02DF165C02EF1000E1C
:1037E000F86E570EF76E180EF66E8AEC0AF0010EA0
:1037F000A0EC06F0B80E8F6F0B0E906F3EEC18F039
:1038000014B228D081EC09F014B224D024EC18F0C2
:10381000F5E2D8EC25F0F2E38B9F31EC18F002E3EF
:103820008B8F18D00101796B7A6B806B816B0001F3
:1038300070EC0AF0000EF86E540EF76EB00EF66ED5
:103840008AEC0AF06FEC02F089EC09F070EC0AF0F7
:10385000D8901200D8801200BADFD8B058EF1DF00F
:10386000626609D0010E766E020E8A6FF5EC15F0D5
:10387000CBEC14F016D0050E626209D0010E776E03
:10388000020E8A6FFBEC15F008EC15F00AD0010E61
:10389000766E010E776E020E8A6F01EC16F030EC38
:1038A00014F073C063F074C064F075C065F0F5EC9B
:1038B00008F0F6EC12F0760E306E050E316EA35164
:1038C000315C02E1A251305CD8B0ACD089D07FDF4E
:1038D000D8B058EF1DF0626609D0010E766E020E68
:1038E0008A6FF8EC15F0CBEC14F016D0050E62627E
:1038F00009D0010E776E020E8A6FFEEC15F008EC0F
:1039000015F00AD0010E766E010E776E010E8A6FE9
:1039100005EC16F030EC14F073C063F074C064F082
:1039200075C065F0F5EC08F0F6EC12F0760E306E2E
:10393000050E316EA351315C02E1A251305CD8B06A
:1039400071D04ED0158601D0159641DFD8B058EF12
:103950001DF0070EA0EC06F089EC09F015A605D0C5
:103960009BEC13F014B27FD004D06FEC13F014B2C0
:103970007AD0F6EC12F079C145F07AC146F07BC1FD
:1039800047F07CC148F07DC149F0A4EC32F0E7EC8F
:1039900033F0D8B033EF1DF03F0E4E6EC00E4D6EBB
:1039A0004A6A4B6A4C6AE7EC33F03CE3010E766EF0
:1039B000010E776E010E8A6F8B9901EC16F030ECD8
:1039C00014F073C063F074C064F075C065F0F5EC7A
:1039D00008F0F6EC12F0080EA0EC06F089EC09F005
:1039E00070EC0AF0000EF86E540EF76EEC0EF66EE8
:1039F0008AEC0AF0000EF86E550EF76E020EF66EA7
:103A00008AEC0AF0020EA0EC06F089EC09F0A9ECB1
:103A10001AF070EC0AF0ADEC1BF036C138F137C18A
:103A200039F146D0080EA0EC06F089EC09F070ECF4
:103A30000AF0000EF86E540EF76EEC0EF66E8AEC7D
:103A40000AF0000EF86E540EF76EC80EF66E8AEC91
:103A50000AF0F6EC12F0030EA0EC06F089EC09F087
:103A6000A9EC1AF025D02CC163F02DC164F02EC151
:103A700065F0F5EC08F0F6EC12F070EC0AF0000ED0
:103A8000F86E540EF76EEC0EF66E8AEC0AF0000E2D
:103A9000F86E540EF76EF80EF66E8AEC0AF0030E0E
:103AA000A0EC06F089EC09F0A9EC1AF048EF1AF046
:103AB0008BBFA9EC1AF070EC0AF0148479EC2CF0AE
:103AC00048EF1AF00101386B396B00011200120047
:103AD00070EF1DF047EC20F0120047EC20F01200D0
:103AE0006EEC0AF070EC0AF0C3EC1DF079520FE0B6
:103AF00079BE06D07A2A0A0E7A6201D07A6A05D097
:103B00007A067AAE02D0090E7A6E796AEDD744EC65
:103B100009F0ECE355EC09F0020E1B6203D039EC1E
:103B20001EF029D0010E1B620BD070EC0AF0000EC3
:103B3000F86E570EF76E2A0EF66E8AEC0AF01BD05E
:103B40000B0E1B620BD070EC0AF0000EF86E570ED5
:103B5000F76E2A0EF66E8AEC0AF00DD00C0E1B6280
:103B60000AD070EC0AF0000EF86E570EF76E2A0EAF
:103B7000F66E8AEC0AF089EC09F070EC0AF0148415
:103B8000796A1B6A1200000EF86E550EF76E3C0E35
:103B9000F66E8AEC0AF07A6608D0000EF86E550EC2
:103BA000F76E4E0EF66E8AEC0AF0010E7A6208D0BD
:103BB000000EF86E550EF76E600EF66E8AEC0AF087
:103BC000020E7A6208D0000EF86E550EF76E720E75
:103BD000F66E8AEC0AF0030E7A6208D0000EF86ED8
:103BE000550EF76E840EF66E8AEC0AF0040E7A62B9
:103BF00008D0000EF86E550EF76E960EF66E8AEC33
:103C00000AF0050E7A6208D0000EF86E550EF76EB7
:103C1000A80EF66E8AEC0AF0060E7A6208D0000E44
:103C2000F86E550EF76EBA0EF66E8AEC0AF0070EB5
:103C30007A6208D0000EF86E550EF76ECC0EF66E56
:103C40008AEC0AF0080E7A6208D0000EF86E550E63
:103C5000F76EDE0EF66E8AEC0AF0090E7A6208D074
:103C6000000EF86E550EF76EF00EF66E8AEC0AF046
:103C7000120070EC0AF07A6602D06DEC1EF0010EB4
:103C80007A6202D077EC1EF0020E7A6202D081ECEA
:103C90001EF0030E7A6202D08BEC1EF0040E7A62E4
:103CA00002D095EC1EF0050E7A6202D09FEC1EF059
:103CB000060E7A6202D0A9EC1EF0070E7A6202D0DC
:103CC000B3EC1EF0080E7A6202D0B5EC1EF0090EBD
:103CD0007A6202D0BFEC1EF01200000EF86E560E93
:103CE000F76EA00EF66E8AEC0AF046EF18F0000EA2
:103CF000F86E560EF76EA80EF66E8AEC0AF044EFD8
:103D000018F0000EF86E560EF76EB40EF66E8AECD2
:103D10000AF0A4EF1CF0000EF86E560EF76EDA0EE5
:103D2000F66E8AEC0AF0A2EF1CF0000EF86E570E49
:103D3000F76E080EF66E8AEC0AF0ADEF1BF0000E7F
:103D4000F86E560EF76EFC0EF66E8AEC0AF0E3EF94
:103D50001BF0000EF86E560EF76EEA0EF66E8AEC49
:103D60000AF09BEF1BF089EF1FF0000EF86E560E65
:103D7000F76EBE0EF66E8AEC0AF02CEF1CF0000E09
:103D8000F86E560EF76ECC0EF66E8AEC0AF067EF00
:103D90001CF070EC0AF0F6EC12F0E9EC01F06BECC0
:103DA0001FF044EC09F014E355EC09F0020E1B621D
:103DB00002D0147EF0D7010E1B6202D05DEC1FF022
:103DC0000B0E1B6201D00CD00C0E1B62E4D708D086
:103DD0007952E1E0F6EC1EF0F5EC08F0796ADBD7F9
:103DE00089EC09F06EEC0AF01B6A120079BE36D03D
:103DF00014BE2BD0666603D0642AD8B4652A010E9F
:103E0000666208D00A0E306E000E316E30506426A5
:103E100031506522020E666208D0640E306E000ECC
:103E2000316E3050642631506522FF0E306E070E21
:103E3000316E6550315C02E16450305CD8B004D022
:103E400030C064F031C065F037D0676601D0632AB6
:103E5000010E676202D00A0E63262ED014BE23D054
:103E6000666606D064066428D8B46506D8B4645281
:103E7000010E666208D00A0E306E000E316E3050B0
:103E8000645E3150655A020E666208D0640E306E70
:103E9000000E316E3050645E3150655A65AE02D00E
:103EA000646A656A09D0676601D06306010E6762BD
:103EB00002D00A0E635E00D0120014BE06D0662A3D
:103EC000030E666201D0666A05D0672A020E676239
:103ED00001D0676A120014BE0ED0666602D0480E8A
:103EE00013D0010E666202D0470E0ED0020E66623B
:103EF00002D0460E09D0676602D0430E05D0010EEF
:103F0000676202D0420E00D078EC0AF06CEC0AF046
:103F100012006EEC0AF070EC0AF0C2EC1FF079525D
:103F20000FE079BE06D0622A060E626201D0626A94
:103F300005D0620662AE02D0050E626E796AEDD7D8
:103F400044EC09F0ECE355EC09F0010E1B6202D0E1
:103F5000F5EC08F0020E1B6202D0F5EC08F00B0E37
:103F60001B620AD0000EF86E570EF76E2A0EF66E20
:103F70008AEC0AF089EC09F070EC0AF01484796A92
:103F80001B6A1200000EF86E540EF76EB80EF66E35
:103F90008AEC0AF087EC2CF062C030F0E9EC36F0E5
:103FA000010E4F6E506ABAEC35F0626610D0000E0A
:103FB000F86E540EF76E800EF66E8AEC0AF0000E64
:103FC000F86E540EF76E840EF66E8AEC0AF0010E4F
:103FD000626210D0000EF86E540EF76E880EF66E08
:103FE0008AEC0AF0000EF86E540EF76E8C0EF66E28
:103FF0008AEC0AF0020E626210D0000EF86E540EC7
:10400000F76E900EF66E8AEC0AF0000EF86E540E03
:10401000F76E940EF66E8AEC0AF0030E626210D010
:10402000000EF86E540EF76E980EF66E8AEC0AF0DB
:10403000000EF86E540EF76E9C0EF66E8AEC0AF0C7
:10404000040E626210D0000EF86E540EF76EA00ED1
:10405000F66E8AEC0AF0000EF86E540EF76EA40E9F
:10406000F66E8AEC0AF0050E626210D0000EF86E51
:10407000540EF76EA80EF66E8AEC0AF0000EF86E7B
:10408000540EF76EAC0EF66E8AEC0AF012006EEC6F
:104090000AF070EC0AF08EEC20F079520FE079BE55
:1040A00006D07B2A100E7B6201D07B6A05D07B068E
:1040B0007BAE02D00F0E7B6E796AEDD744EC09F02F
:1040C000ECE355EC09F0020E1B6203D046EC21F044
:1040D0001DD0010E1B6203D046EC21F017D00B0E51
:1040E0001B6209D0000EF86E570EF76E2A0EF66EA0
:1040F0008AEC0AF00BD00C0E1B6208D0000EF86E92
:10410000570EF76E2A0EF66E8AEC0AF089EC09F06B
:1041100070EC0AF01484796A1B6A1200000EF86EC3
:10412000500EF76EE60EF66E8AEC0AF07B6608D04B
:10413000000EF86E500EF76EF80EF66E8AEC0AF06E
:10414000010E7B6208D0000EF86E510EF76E0A0E5B
:10415000F66E8AEC0AF0020E7B6208D0000EF86E52
:10416000510EF76E1C0EF66E8AEC0AF0030E7B629F
:1041700008D0000EF86E510EF76E2E0EF66E8AEC19
:104180000AF0040E7B6208D0000EF86E510EF76E36
:10419000400EF66E8AEC0AF0050E7B6208D0000E27
:1041A000F86E510EF76E520EF66E8AEC0AF0060E9D
:1041B0007B6208D0000EF86E510EF76E640EF66E3C
:1041C0008AEC0AF0070E7B6208D0000EF86E510EE2
:1041D000F76E760EF66E8AEC0AF0080E7B6208D057
:1041E000000EF86E510EF76E9A0EF66E8AEC0AF01B
:1041F000090E7B6208D0000EF86E510EF76EAC0E01
:10420000F66E8AEC0AF00A0E7B6208D0000EF86E99
:10421000510EF76EBE0EF66E8AEC0AF00B0E7B6244
:1042200008D0000EF86E510EF76ED80EF66E8AECBE
:104230000AF00C0E7B6208D0000EF86E510EF76E7D
:10424000FA0EF66E8AEC0AF00D0E7B6208D0000EB4
:10425000F86E530EF76EC20EF66E8AEC0AF00E0E72
:104260007B6208D0000EF86E530EF76EE00EF66E0D
:104270008AEC0AF00F0E7B6208D0000EF86E530E27
:10428000F76EF20EF66E8AEC0AF012007B6600D032
:10429000010E7B6202D0DCEC24F0020E7B6202D0C5
:1042A000F3EC0FF0030E7B6202D0F1EC0FF0040E82
:1042B0007B6202D061EC25F0050E7B6202D017EC28
:1042C00003F0060E7B6202D022EC03F0070E7B6245
:1042D00002D091EC23F0080E7B6202D09BEC0FF031
:1042E000090E7B6202D0AFEC0FF00A0E7B6202D0A7
:1042F00094EC21F00B0E7B6202D02EEC22F00C0E1F
:104300007B6202D02AEC23F00D0E7B6202D0E4EC3B
:1043100022F00E0E7B6202D030EC26F00F0E7B6294
:1043200002D0B7EC22F0120070EC0AF08CEC09F02D
:10433000D7EC11F010EC01F03FEC01F03AC145F080
:104340003BC146F03CC147F03DC148F03EC149F099
:10435000CFEC00F046EC31F045C03AF146C03BF1FD
:1043600047C03CF148C03DF149C03EF141C145F074
:1043700042C146F043C147F044C148F045C149F04D
:10438000CFEC00F046EC31F045C041F146C042F1BF
:1043900047C043F148C044F149C045F1000EF86EF2
:1043A000510EF76ED00EF66E8AEC0AF03AC145F067
:1043B0003BC146F03CC147F03DC148F03EC149F029
:1043C00012EC22F07AEC0AF079EC2CF096C030F086
:1043D00097C031F026EC22F0000EF86E510EF76E09
:1043E000D40EF66E8AEC0AF041C145F042C146F0A7
:1043F00043C147F044C148F045C149F012EC22F0F6
:104400007AEC0AF079EC2CF098C030F099C031F0D9
:1044100026EC22F044EC09F002E296EF21F055EC94
:1044200009F0120002EC37F0030E4F6E010E506ED1
:104430005284A3EC36F0E6EC35F0000EF86E580E20
:10444000F76EE60EF66E8DEC0AF01200E9EC36F02F
:10445000050E4F6E506ABAEC35F0120070EC0AF09F
:10446000000EF86E510EF76EEA0EF66E8AEC0AF048
:1044700087EC2CF0A9C030F0E9EC36F0020E4F6E5C
:10448000BAEC35F0000EF86E580EF76EE60EF66ECA
:104490008DEC0AF07AEC0AF087EC2CF0A9C030F031
:1044A000F4EC2EF040C04BF241C04CF242C04DF251
:1044B00043C04EF244C04FF25EEC38F0D3EC38F01B
:1044C00050EC3BF0AA51DAEC00F0000EF86E510E01
:1044D000F76EF00EF66E8AEC0AF087EC2CF0ABC0AB
:1044E00030F0ACC031F0E9EC36F0050E4F6EBAECAE
:1044F00035F0795206E079AEA92B79BEA907796A21
:10450000AFD744EC09F0F5E355EC09F0020E1B625D
:1045100005D0DAEC00F04FEC11F000D091EC22F075
:104520001200000EF86E540EF76E320EF66E8AEC24
:104530000AF087EC2CF0ABC030F0ACC031F0E9EC05
:1045400036F0BAEC35F0000EF86E540EF76E3C0EF5
:10455000F66E8AEC0AF087EC2CF0ADC030F0AEC0FD
:1045600031F0E9EC36F0BAEC35F089EF09F070EC97
:104570000AF0000EF86E530EF76ED40EF66E8AEC4B
:104580000AF07C503009E7EC09F0795212E079BE6C
:1045900007D07C2A050E7C6402D0010E7C6E07D009
:1045A0007C067CBE02D07C6602D0050E7C6E796AE9
:1045B000E0D744EC09F0E9E355EC09F0020E1B6288
:1045C00002D027EC11F0120070EC0AF07CC07DF0F4
:1045D000000EF86E530EF76ED40EF66E8AEC0AF0EB
:1045E0007D503009E7EC09F0795212E079BE07D02E
:1045F0007D2A050E7D6402D0010E7D6E07D07D06FA
:104600007DBE02D07D6602D0050E7D6E796AE0D750
:1046100044EC09F0E9E355EC09F0020E1B6219D0F5
:10462000010E7D6202D01BEF27F0020E7D6202D0E8
:104630002EEF27F0030E7D6202D041EF27F0040E2B
:104640007D6202D054EF27F0050E7D6202D067EF45
:1046500027F0120070EC0AF0000EF86E520EF76EA2
:104660000C0EF66E8AEC0AF087EC2CF0AAC030F043
:10467000E9EC36F0020E4F6EBAEC35F0000EF86E33
:10468000580EF76EE60EF66E8DEC0AF07AEC0AF034
:1046900087EC2CF0AAC030F0F4EC2EF040C04BF2C6
:1046A00041C04CF242C04DF243C04EF244C04FF202
:1046B0005EEC38F0D3EC38F050EC3BF0AA51DAEC79
:1046C00000F0000EF86E510EF76EF00EF66E8AECEA
:1046D0000AF087EC2CF0ADC030F0AEC031F0E9EC60
:1046E00036F0050E4F6EBAEC35F0795206E079AE31
:1046F000AA2B79BEAA07796AAFD744EC09F0F5E393
:1047000055EC09F0020E1B6205D0DAEC00F03DEC2E
:1047100011F000D091EC22F012005F6A606A616AC9
:10472000120070EC0AF0F9DF0E6AB1EC23F0795058
:1047300010E079BE07D00E2A180E0E6201D00E6A64
:10474000796AF3D70E060EAE02D0170E0E6E796A96
:10475000ECD744EC09F0EBE355EC09F0F5EC08F08C
:104760001200000EF86E510EF76E880EF66E8AEC8F
:104770000AF0D3DF0E6609D0000EF86E520EF76E07
:10478000120EF66E8AEC0AF06180010E0E6209D0FC
:10479000000EF86E520EF76E240EF66E8AEC0AF0DA
:1047A0006182020E0E6209D0000EF86E520EF76E94
:1047B000360EF66E8AEC0AF06184030E0E6209D0A2
:1047C000000EF86E520EF76E480EF66E8AEC0AF086
:1047D0006186040E0E6209D0000EF86E520EF76E5E
:1047E0005A0EF66E8AEC0AF06188050E0E6209D048
:1047F000000EF86E520EF76E6C0EF66E8AEC0AF032
:10480000618A060E0E6209D0000EF86E520EF76E27
:104810007E0EF66E8AEC0AF0618C070E0E6209D0ED
:10482000000EF86E520EF76E900EF66E8AEC0AF0DD
:10483000618E080E0E6209D0000EF86E520EF76EF1
:10484000A20EF66E8AEC0AF06080090E0E6209D0A4
:10485000000EF86E520EF76EB40EF66E8AEC0AF089
:1048600060820A0E0E6209D0000EF86E520EF76ECC
:10487000C60EF66E8AEC0AF060840B0E0E6209D04A
:10488000000EF86E520EF76ED80EF66E8AEC0AF035
:1048900060860C0E0E6209D0000EF86E520EF76E96
:1048A000EA0EF66E8AEC0AF060880D0E0E6209D0F0
:1048B000000EF86E520EF76EFC0EF66E8AEC0AF0E1
:1048C000608A0E0E0E6209D0000EF86E530EF76E5F
:1048D0000E0EF66E8AEC0AF0608C0F0E0E6209D096
:1048E000000EF86E530EF76E200EF66E8AEC0AF08C
:1048F000608E100E0E6209D0000EF86E530EF76E29
:10490000320EF66E8AEC0AF05F80110E0E6209D04C
:10491000000EF86E530EF76E440EF66E8AEC0AF037
:104920005F82120E0E6209D0000EF86E530EF76E03
:10493000560EF66E8AEC0AF05F84130E0E6209D0F2
:10494000000EF86E530EF76E680EF66E8AEC0AF0E3
:104950005F86140E0E6209D0000EF86E530EF76ECD
:104960007A0EF66E8AEC0AF05F88150E0E6209D098
:10497000000EF86E530EF76E8C0EF66E8AEC0AF08F
:104980005F8A160E0E6209D0000EF86E530EF76E97
:104990009E0EF66E8AEC0AF05F8C170E0E6209D03E
:1049A000000EF86E530EF76EB00EF66E8AEC0AF03B
:1049B0005F8E1FEC09F0120070EC0AF0D7EC11F0DA
:1049C00010EC01F03FEC01F023EC00F098EC00F06B
:1049D000000EF86E540EF76E5E0EF66E8AEC0AF05C
:1049E0003AC145F03BC146F03CC147F03DC148F0FB
:1049F0003EC149F002EC37F0040E4F6E020E506ECD
:104A0000A3EC36F05284E6EC35F0000EF86E540E4E
:104A1000F76E620EF66E8AEC0AF09DC045F09EC0FD
:104A200046F09FC047F0A0C048F0A1C049F002EC9A
:104A300037F0050E4F6E030E506EA3EC36F0E6EC29
:104A400035F0000EF86E540EF76E660EF66E8AECB8
:104A50000AF041C145F042C146F043C147F044C1AC
:104A600048F045C149F002EC37F0040E4F6E020EDB
:104A7000506EA3EC36F05284E6EC35F0000EF86E82
:104A8000540EF76E6A0EF66E8AEC0AF046C145F0D7
:104A900047C146F048C147F049C148F04AC149F012
:104AA00002EC37F0040E4F6E020E506EA3EC36F09F
:104AB000E6EC35F08DEC09F044EC09F0D8A07ED797
:104AC000120070EC0AF00AEC0CF0000E78EC0AF020
:104AD00079EC2CF057C030F058C031F059C032F0AA
:104AE000E9EC36F0060E4F6E040E506EBAEC35F05F
:104AF000000EF86E540EF76EC40EF66E8DEC0AF0D2
:104B0000000EF86E560EF76E7A0EF66E8AEC0AF00C
:104B10005AC030F0D7EC2EF073EC30F002EC37F0E6
:104B2000030E4F6E506A5284E6EC35F0000EF86EBC
:104B3000560EF76E820EF66E8AEC0AF0000EF86ED4
:104B4000560EF76E880EF66E8AEC0AF08DEC09F0C0
:104B5000795206E079BE5A2A79AE5A06796AB3D7F5
:104B600044EC09F0B0E355EC09F0020E1B620FD0E3
:104B700070EC0AF085EC11F0000EF86E560EF76E30
:104B80008E0EF66E8AEC0AF089EC09F010D0010E58
:104B90001B620DD070EC0AF0000EF86E570EF76E27
:104BA0002A0EF66E8AEC0AF089EC09F000D01200A9
:104BB00000EC0CF02AE355C0A6F056C0A7F00AECB2
:104BC0000CF05650A75D02E15550A65DD8B41FD039
:104BD000A62BD8B4A72B5650A75D02E15550A65D71
:104BE000D8B415D0A607A629D8B4A707D8B4A65319
:104BF000A607A629D8B4A707D8B4A6535650A75DD0
:104C000002E15550A65DD8B402D0D89010D055C05E
:104C100034F156C035F115BE05D034C136F135C179
:104C200037F104D036C134F137C135F1D8801200E4
:104C300030503009E7EC09F01200795210E079AEFB
:104C400006D03006306602D0050E306E07D0302A0E
:104C5000050E306402D0010E306E796AD8941200CD
:104C600070EC0AF0000EF86E560EF76E020EF66E3D
:104C70008AEC0AF052EC09F07CC030F0000EF86EBD
:104C8000560EF76E0E0EF66E8AEC0AF0D1DFD5DF07
:104C9000F5E144EC09F0FBE355EC09F0020E1B6270
:104CA00017D030C035F01B6A000EF86E560EF76E46
:104CB000180EF66E8AEC0AF0BBDFBFDFF5E144ECBC
:104CC00009F0FBE355EC09F0020E1B6201D001D0A4
:104CD000120070EC0AF030C036F03650355CD8B4B3
:104CE00021D0000EF86E560EF76E020EF66E8AECAC
:104CF0000AF035C0E8FF3009E7EC09F036C0E8FFFC
:104D00003009E7EC09F035C030F06CD830C07EF0E7
:104D100031C07FF036C030F065D830C080F031C08F
:104D200081F005D889EC09F01B6A796A1200880EB7
:104D3000306E2C0E316EEDEC2EF040C00EF241C004
:104D40000FF242C010F243C011F244C012F2846B61
:104D5000856B836B000EF86E540EF76E040EF66EC4
:104D60008AEC0AF0D2EC27F002EC37F0030E4F6E1B
:104D7000506AA3EC36F0E6EC35F0000EF86E580EF3
:104D8000F76E260EF66E8DEC0AF08351825DD8B474
:104D900006D082C0E8FF18EC07F082C083F07EC026
:104DA00008F07FC009F0B3EC0BF00AC00BF080C034
:104DB00008F081C009F0AEEC0BF07E2AD8B47F2A4F
:104DC000802BD8B4812B842BD8B4852B880E306EE1
:104DD0002C0E316E8551315C02E18451305CD8A4D7
:104DE000B9D71200010E306205D0000E306E000EF1
:104DF000316E20D0020E306205D0880E306E2C0E3F
:104E0000316E18D0030E306205D0100E306E590E80
:104E1000316E10D0040E306205D0980E306E850EC3
:104E2000316E08D0050E306205D0200E306EB20E05
:104E3000316E00D0120070EC0AF0000EF86E560EC3
:104E4000F76E220EF66E8AEC0AF0000E7E6E000EF1
:104E50007F6E880E806F2C0E816F4BD070EC0AF045
:104E6000000EF86E560EF76E320EF66E8AEC0AF0F1
:104E7000880E7E6E2C0E7F6E100E806F590E816F25
:104E800038D070EC0AF0000EF86E560EF76E420E37
:104E9000F66E8AEC0AF0100E7E6E590E7F6E980E3A
:104EA000806F850E816F25D070EC0AF0000EF86ED1
:104EB000560EF76E520EF66E8AEC0AF0980E7E6E63
:104EC000850E7F6E200E806FB20E816F12D070EC57
:104ED0000AF0000EF86E560EF76E620EF66E8AEC51
:104EE0000AF0200E7E6EB20E7F6EA80E806FDE0E70
:104EF000816F0B68880E306E2C0E316EEDEC2EF04B
:104F000040C00EF241C00FF242C010F243C011F295
:104F100044C012F2846B856B836B000EF86E560EE4
:104F2000F76E720EF66E8AEC0AF07EC030F07FC02B
:104F300031F0315081EC0AF0305081EC0AF07AEC1B
:104F40000AF0D2EC27F002EC37F0030E4F6E506AF5
:104F5000A3EC36F0E6EC35F0000EF86E580EF76E66
:104F6000260EF66E8DEC0AF08351825DD8B406D021
:104F700082C0E8FF18EC07F082C083F0842BD8B41D
:104F8000852B7EC008F07FC009F0AEEC0BF07E2AC6
:104F9000D8B47F2A81517F5C02E180517E5CD8A425
:104FA000BCD7120084C030F085C031F0EDEC2EF09B
:104FB00073EC30F09AEC2CF009EC31F049EC33F062
:104FC00019EC2EF026C082F01200000EF86E500E82
:104FD000F76EC20EF66E8AEC0AF01200000EF86E42
:104FE000500EF76ED40EF66E8AEC0AF01200EACF7D
:104FF00004F0E9CF03F0B0C0EAFFAFC0E9FF9EAA1A
:105000000ED0AE50ABA204D0AE50AB98AB88F7D761
:10501000EE6EF10EE95C02E105EE00F0F0D7EACFAA
:10502000B0F0E9CFAFF0F2A402D0F2943AD0F2A2FD
:1050300006D0F29281B2792A81A2790632D09EA05E
:1050400024D015A002D0929A15908D678D07916794
:1050500091078E678E07906702D08F5306E08F0707
:105060008F29D8B49007D8B48F53936702D0925346
:1050700006E092079229D8B49307D8B49253000E51
:10508000CE6ED30ECF6E9E900CD09EA202D09E927A
:1050900008D0F0A002D0F09004D0A1A202D0A1923A
:1050A00000D004C0EAFF03C0E9FF1100006ED8CFB2
:1050B00001F0E0CF02F002C0E0FF005001C0D8FFD5
:1050C0001000002020202020202020202020202030
:1050D00020202000402020202020202020202020D0
:1050E000202020202000003D3D3D3D2053455455CB
:1050F00050203D3D3D3D3D00404162627275636818
:1051000021202020202020202000404D4B2E5265C1
:105110007475726E204C6F7373202000404B616C6D
:1051200069622E20566F726C617566202000404BBC
:10513000616C69622E20527565636B6C61756600E7
:10514000404B616C69622E4F66667365742D4672C2
:1051500071004056696577204D4B787920566F7203
:10516000202020004056696577204D4B78792052E9
:105170007565636B20004052656C6169732D5465E1
:105180007374202020202000002D2D2D2D2052650D
:105190006C616973202D2D2D2D00404B616C2E6D9F
:1051A000616E75656C6C20566F722000404B616CAF
:1051B0002E6D616E2E202020527565636B00405667
:1051C0006965772064426D2B412F442C562B520089
:1051D00000563A0040523A00405365742064426DD4
:1051E000204D696E696D756D2000004D696E3A0045
:1051F0004041442D576572743A00405365742064F1
:10520000426D204D6178696D756D2000004D6178AB
:105210003A00404B4C31204C2D476C2E32204A3105
:105220002F352000404B4C32204C2D476C2E322025
:105230004A312F362000404B4C33204C2D476C2EEA
:1052400032204A312F372000404B4C34204C2D4720
:105250006C2E32204A312F382000404B4C35204CE8
:105260002D476C2E31204A312F382000404B4C36D0
:10527000204C2D476C2E31204A312F372000404BD7
:105280004C37204C2D476C2E31204A312F362000D0
:10529000404B4C38204C2D476C2E31204A312F3555
:1052A0002000404B433120432D476C2E20204A31B3
:1052B0002F362000404B433220432D476C2E2020B8
:1052C0004A312F352000404B433320432D476C2E6D
:1052D00020204A312F342000404B433420432D47B7
:1052E0006C2E20204A312F332000404B4335204381
:1052F0002D476C2E20204A312F322000404B433660
:1053000020432D476C2E20204A312F312000404B66
:10531000433720432D476C2E20204A322F31200066
:10532000404B433820432D476C2E20204A322F32E9
:105330002000404B433920432D476C2E20204A3219
:105340002F332000404B43313020432D476C2E201B
:105350004A322F342000404B43313120432D476CDB
:105360002E204A322F3520004066726569202020A9
:1053700020202020202020202000404B4C433120A2
:105380004C2D476C2E32204A312F3400404B4C4379
:1053900032204C2D476C2E32204A312F3300404BA7
:1053A0004C4333204C2D476C2E31204A312F340092
:1053B000404B4C4334204C2D476C2E31204A312F2A
:1053C000330040416E74656E6E6520436C6561729A
:1053D0002020200000416E74656E6E65233A000047
:1053E00040416E74656E6E6520436F707920202099
:1053F000200040416E74656E6E652073656C656358
:10540000742020004050726F67726573733A000019
:10541000002D2D2D205049432D5761746368646F12
:1054200067202D2D2D004052657374617274733A9C
:105430000000004144436D696E3A0000404144431E
:105440006D61783A00000041444320203064426D91
:105450003A00404144432D333064426D3A000056D7
:105460000000085300004052000048524C004054D5
:1054700061737465206C616E6721202020202000FC
:105480000E2D4C004E2020000E4C2B004E204300D1
:105490000E2B4C004E4320000E432B004E204C00A0
:1054A0000E2B43004E4C20000E2D43004E202000BA
:1054B000004672713A200000404C2F432D56617215
:1054C0003A2000004D487A00406E6963687473208A
:1054D000676566756E64656E2100404B65696E2078
:1054E00053656E64657369676E616C000041627339
:1054F00074696D6D756E67004041626272756368B4
:105500002100404F4B20212100000053617665208F
:105510006578742E456570726F6D2100005265616B
:105520006479210000416E74656E6E653A2000005A
:1055300000536176652042616E642100002D2D2D9F
:10554000204D656E75202D2D2D20204F4B00404D98
:105550006174636820202020202020202020580013
:10556000404D6174636820646565702020202020B0
:1055700058004052654D617463682020202020202F
:10558000202058004052654D617463682064656551
:105590007020202058004031306B487A20536567D6
:1055A0006D656E74202058004042616E6420736106
:1055B0007665202020202020580040535752205745
:1055C000617474202020202020205800404C432D5E
:1055D00056617269616E7465202020205800405227
:1055E000654D617463682034783420202020580091
:1055F0004052654D6174636820387838202020203F
:10560000580000416E742E20636F70793A0040514B
:1056100075656C6C653A0000405A69656C20203AEB
:10562000000000416E74656E6E65203120434C525F
:10563000000000416E74656E6E65203220434C524E
:10564000000000416E74656E6E65203320434C523D
:10565000000000416E74656E6E65203420434C522C
:10566000000000416E74656E6E65203520434C521B
:10567000000040414444523A200040546F66663A6C
:1056800000000C2B204F4B004C2D20205800405484
:105690006F722D4F666673657420536176652100C5
:1056A000004D617463680000004D617463682044BC
:1056B000656570000052652D4D617463680000528D
:1056C000652D4D6174636820347834000052652D77
:1056D0004D6174636820387838000052652D4D6143
:1056E00074636820446565700000005357520000E1
:1056F000005A20496D706564616E7A000042616EE7
:1057000064207361766500000031304B687A207345
:1057100061766500004A61004057617274656E20D1
:1057200054582120202020202000404162627275C0
:10573000636820212121202020202000004B656962
:105740006E65204672657175656E7A2D2000406920
:105750006E666F726D6174696F6E2021212020006A
:1057600000566F726C617566202020202020204F2B
:105770004B0000527565636B6C61756620202020BC
:10578000204F4B004F5800004020203064426D3ABB
:1057900000000020203064426D3A0000402D33307C
:1057A00064426D3A0000006B783A0000406B793A31
:1057B0000000004B616C696272696572756E6720EA
:1057C000204F4B00405370656963682E2020416272
:1057D000627275636800004265737461657469671D
:1057E000756E672020202000004C432D56617269A1
:1057F000616E7465203D200003533A0040535752B8
:105800003A000053746570204C3A00000B433A0094
:10581000024C3A00402020433A0075480000706670
:1058200000006E660000250002207C5A7C3A0000D1
:10583000003D3D205361766520446174656E203DD6
:105840003D00403D3D2050494320456570726F6DDD
:10585000203D3D00003D3D3D3D2050696341545594
:10586000203D3D3D3D00403D3D3D3D20536C656547
:1058700070203D3D3D3D3D00005069634154552041
:10588000203530302057617474004056312E313548
:1058900020202030372E31312E323200404857310F
:1058A0002E303220286329444C344A414C002D2D9F
:1058B0002D00494E46006D570000755700006E5789
:1058C0000000705700006657000061570000572025
:1058D00000006B570000205600006D560000755602
:1058E00000006E56000064426D0064420000737355
:1058F000000013D806D82B6A2C6A2D6A2E6A2F6AEC
:105900001200266A276A286A296A2A6A1200306AFF
:10591000316A326A336A346A1200F9DF356A366AEC
:10592000376A386A396A1200456A466A476A486ABD
:10593000496A12000EC24AF00FC24BF010C24CF07E
:1059400011C24DF012C24EF012000EC245F00FC24D
:1059500046F010C247F011C248F012C249F01200DE
:105960004AC045F04BC046F04CC047F04DC048F02F
:105970004EC049F0120045C04AF046C04BF047C047
:105980004CF048C04DF049C04EF0120045C00EF238
:1059900046C00FF247C010F248C011F249C012F2DF
:1059A000120013C245F014C246F015C247F016C2E9
:1059B00048F017C249F0120013C24AF014C24BF06B
:1059C00015C24CF016C24DF017C24EF0120018C2AC
:1059D00045F019C246F01AC247F01BC248F01CC27B
:1059E00049F0120018C24AF019C24BF01AC24CF02A
:1059F0001BC24DF01CC24EF012001DC245F01EC26B
:105A000046F01FC247F020C248F021C249F0120000
:105A10001DC24AF01EC24BF01FC24CF020C24DF016
:105A200021C24EF0120022C245F023C246F024C229
:105A300047F025C248F026C249F0120022C24AF0BF
:105A400023C24BF024C24CF025C24DF026C24EF0CA
:105A5000120027C245F028C246F029C247F02AC2E8
:105A600048F02BC249F0120027C24AF028C24BF07E
:105A700029C24CF02AC24DF02BC24EF012004AC08F
:105A800013F24BC014F24CC015F24DC016F24EC0CA
:105A900017F2120045C013F246C014F247C015F2C7
:105AA00048C016F249C017F2120045C018F246C0AD
:105AB00019F247C01AF248C01BF249C01CF212008A
:105AC00045C01DF246C01EF247C01FF248C020F27A
:105AD00049C021F2120045C022F246C023F247C05D
:105AE00024F248C025F249C026F2120045C027F230
:105AF00046C028F247C029F248C02AF249C02BF21A
:105B0000120026C030F027C031F028C032F029C082
:105B100033F02AC034F0120026C035F027C036F02A
:105B200028C037F029C038F02AC039F0120030C040
:105B300026F031C027F032C028F033C029F034C03D
:105B40002AF01200353636363736383639361200F6
:105B50003036313632363336343612003932383256
:105B60003732363235321200343233323232313259
:105B70003032120006D82B362C362D362E362F36E4
:105B8000120026362736283629362A3612002F32BA
:105B90002E322D322C322B321200F9DF2A322932EA
:105BA000283227322632120030AE04D031683268F3
:105BB00033683468120031AE03D032683368346819
:105BC000120032AE02D033683468120033AE01D016
:105BD00034681200539252BE53828CDE280E236E1C
:105BE000D890B4EC2DF0CEEC2DF003D8232EF8D7BE
:105BF0001200CEEC37F00A0E226E00EE26F0EF50C7
:105C0000E8B6FD0FE8BED00FEE6E222EF8D7DBEC23
:105C100037F012003FD82AAE09D02B2AD8B42C2A4C
:105C2000D8B42D2AD8B42E2AD8B42F2A81EC2CF03F
:105C300035D030D82AAE09D02B2AD8B42C2AD8B4E3
:105C40002D2AD8B42E2AD8B42F2A2BC026F02CC047
:105C500027F02DC028F02EC029F02FC02AF052BE08
:105C6000C2EC34F0120016D82BC026F02CC027F05E
:105C70002DC028F02EC029F02FC02AF052BEC2EC51
:105C800034F0120007D87BEC2CF008D003D881EC5C
:105C90002CF004D05DEC30F052EF2EF00FEC2FF032
:105CA00073EF30F04CD803E17AEC2CF01AD01AD80C
:105CB0007F0E3A6E3A503E5E3B503F5A3EC022F055
:105CC0003E520FE03EBE06D0D890BAEC2DF0222E08
:105CD000FBD707D0221E222AD890CDEC2DF0222E01
:105CE000FBD71200529E44BE528E449E7AEC2CF09A
:105CF00040C027F041C028F042C029F043C02AF03C
:105D000044C02BF0D890BAEC2DF0CEEC2DF02A8EBA
:105D10002BC03EF02B6AD890BAEC2DF01200040E86
:105D2000226EEE6608D0222EFCD7EECFE8FF7F0B66
:105D300003E1D88401D0D894DBEC37F01200CEEC2C
:105D400037F000EE40F0EBD7CEEC37F000EE45F048
:105D5000E6D7CEEC37F000EE4AF0E1D7CEEC37F0E4
:105D600000EE30F0DCD7CEEC37F000EE35F0D7D7D0
:105D7000CEEC37F000EE26F00A0E226EEE66DBD790
:105D8000222EFCD7D6D7346A33BE346835D0336A76
:105D9000346A32AE31D0336834682ED0326A336A16
:105DA000346A31AE29D032683368346825D0316A1C
:105DB000326A336A346A30AE1FD031683268336871
:105DC00034681AD07AEC2CF0529E346A1DD07AECEA
:105DD0002CF0529E336A346A17D07AEC2CF0529E23
:105DE000326A336A346A10D07AEC2CF0529E316AEF
:105DF000326A336A346A08D07AEC2CF0529E34AEA0
:105E000003D0D1EC34F0528E30C02BF031C02CF0E6
:105E100032C02DF033C02EF034C02FF000D07F0EF2
:105E20003E6E000E3F6EB8EC2EF006E1406A416A0D
:105E3000426A436A446A36D079EC2FF007E0D89082
:105E4000CDEC2DF03E2AD8B43F2AF6D72BB00AD09D
:105E5000D890BAEC2DF03E063E28D8B43F06D8B410
:105E60003E52F4D727A00BD02780272AD8B4282A5F
:105E7000D8B4292AD8B42A2AD8B42B2ADDD7266A3E
:105E80002B903EC02BF0CDEC2DF027C040F028C069
:105E900041F029C042F02AC043F02BC044F0449E98
:105EA00052BE448E1200406A416A426A446A800EC1
:105EB000436EF5D74068416842687F0E436E7F0E9F
:105EC000446EEDD77F0E306E000E316E3F50315C68
:105ED00002E13E50305CD8B003D0ECDFD88401D072
:105EE000D89412003FAE03D0DEDFD88401D0D8941E
:105EF0001200CEEC37F000EE2FF0040E226EED66AD
:105F00000AD0222EFCD7010EEF6201D002D0EF663C
:105F100002D0D88401D0D894DBEC37F0120035C021
:105F200000F236C001F237C002F238C003F239C0C5
:105F300004F2D9EC2FF026C007F227C008F228C0DF
:105F400009F229C00AF22AC00BF200C230F001C2E5
:105F500031F002C232F003C233F004C234F0BFECBD
:105F60002FF007C22BF008C22CF009C22DF00AC294
:105F70002EF00BC22FF0529E53B2528E1200BADC9A
:105F8000280E236ED89005D8C1EC2DF0232EFAD719
:105F90001200CEEC37F0050E226E00EE30F0D890F5
:105FA000EF50E8200700EE6E222EFAD7DBEC37F038
:105FB0001200CEEC37F09EDC280E236ED890B4ECA5
:105FC0002DF0CEEC2DF000EE30F0050E226EEFAE8F
:105FD00002D0300EEF5EEFA602D0030EEF5EEE525F
:105FE000222EF5D7232EEAD7DBEC37F0120002D8A9
:105FF00081EF2DF0CEEC37F09ADD00EE26F010EEBA
:1060000035F0040E226EE650EE5EE650EE5A222E79
:10601000FCD7DBEC37F0120002D881EF2DF0CEEC8C
:1060200037F085DD00EE26F010EE35F0E650EE2676
:10603000040E226EE650EE22222EFCD7DBEC37F067
:10604000120000C230F001C231F002C232F003C2CD
:1060500033F004C234F005C23AF006C23BF012003D
:1060600007C235F008C236F009C237F00AC238F06C
:106070000BC239F00CC23CF00DC23DF0120027C03B
:1060800000F228C001F229C002F22AC003F22BC09C
:1060900004F23EC005F23FC006F2120027C007F22C
:1060A00028C008F229C009F22AC00AF22BC00BF25C
:1060B0003EC00CF23FC00DF2120045C040F046C099
:1060C00041F047C042F048C043F049C044F01200DC
:1060D0004AC040F04BC041F04CC042F04DC043F0CC
:1060E0004EC044F0120040C045F041C046F042C0EE
:1060F00047F043C048F044C049F0120040C04AF0A5
:1061000041C04BF042C04CF043C04DF044C04EF093
:106110001200EBEC37F016E2E8EC37F013E2A4ECF7
:106120002EF01AE0A9EC2EF017E000EC38F004E3B2
:10613000A4EC2EF001E306D003EC38F006E3A9EC62
:106140002EF003E328EC38F0120000EC38F003E303
:106150001DEC38F003D00DD094EC2CF049BE03D0E8
:106160004EAE01D0498E49AE03D04EBE01D0498E0D
:1061700012001DD8529E52BA527E52BC527E7EEC04
:1061800034F02AC000F22BC001F22CC002F22DC064
:1061900003F22EC004F21ED80FEC30F081EC2DF08B
:1061A0008EEC2CF07F0E356EFAEC2FF01ED0529A4A
:1061B000529C49BE528A4EBE528C7FDF72EC2EF04A
:1061C0005EDF86DF72EC2EF069DF79EC2CF039DFD0
:1061D00030EF30F079EC2CF03AC030F03BC031F0C9
:1061E0003CC035F03DC036F0120026C03EF027C05E
:1061F0003FF07AEC2CF000C227F001C228F002C276
:1062000029F003C22AF004C22BF013EC2FF073EF35
:1062100030F0EBEC37F009E2E8EC37F006E2A4EC02
:106220002EF006E1A9EC2EF019E128EC38F012006E
:1062300003EC38F003E300EC38F0F7E2A9EC2EF0C1
:1062400010E11DEC38F049BE03D04EAE01D0498EAE
:1062500049AE03D04EBE01D0498E120032EC38F068
:10626000F2D7A5DF529E52BA527E52BC527E4CECFF
:1062700035F005DFAFDFFAEC2FF081EC2DF08EEC7E
:106280002CF07F0E356E0FEC30F0AFD7A9EC2EF06E
:1062900001E112004E7E00D0EBEC37F004E2E8ECB6
:1062A00037F001E203D028EC38F01200A9EC2EF010
:1062B00001E11200A4EC2EF003E1B0EC2CF012008E
:1062C00017D80FEC30F03AC03EF03BC03FF0529E82
:1062D0002AAE03D0528EC2EC34F026C000F227C0A2
:1062E00001F228C002F229C003F22AC004F281D7C9
:1062F0005EDFFE0E3E6E000E3F6E3D503B5C02E1E7
:106300003C503A5C27E013E33C2AD8B43D2A3F5086
:106310003D5C02E13E503C5C07E18EEC2CF03AC063
:106320003CF03BC03DF016D0D89018DCE6D73A2AB6
:10633000D8B43B2A3F503B5C02E13E503A5C07E157
:1063400087EC2CF03CC03AF03DC03BF003D0D89035
:106350000BDCD3D752BAD1EC34F052BCE0EC34F0C1
:106360001200BBEC2CF089EF30F0A4EC2EF02DE005
:1063700049BE2CD0EBEC37F028E2C6EC2CF0ECD880
:1063800048DF4AEC2DF01E0E256E254E1ED0A5ECE2
:106390002CF0DCEC2CF03DDFDCEC2CF07DDFDCD8ED
:1063A00038DFDCEC2CF04E50495C0BE14D50485C82
:1063B00008E14C50475C05E14B50465C02E14A5015
:1063C000455C03E04AEC2DF0E0D7120028EC38F0F1
:1063D0001200A4EC2EF008E13F0E496E800E486ECC
:1063E000456A466A476A120002013F0E266F800E18
:1063F000256F226B236B246B3F0E216F800E206F65
:106400001D6B1E6B1F6B000155EC2DF04AEC2DF03F
:1064100022C20EF223C20FF224C210F225C211F2E0
:1064200026C212F21E0E256ED1EC2CF008EC2DF0D7
:10643000F0DE9AEC2CF04CEC31F09AEC2CF04E5053
:10644000495C0BE14D50485C08E14C50475C05E16C
:106450004B50465C02E14A50455C17E0254E15D092
:10646000C6EC2CF013EC2DF06FD816DF6BEC2DF092
:1064700008EC2DF04EDE60EC2DF0E7EC2CF0DCECBF
:106480002CF047DE4AEC2DF0CFD71200A4EC2EF012
:1064900008E13F0E496E800E486E456A466A476ABB
:1064A000120045C02CF246C02DF247C02EF248C063
:1064B0002FF249C030F242EC2EF03BD82ADE89DFC1
:1064C00076EC2DF02CC245F02DC246F02EC247F0DE
:1064D0002FC248F030C249F04AEC2EF0529452BE1E
:1064E00052842BC025F027C245F028C246F029C2AD
:1064F00047F02AC248F02BC249F0255206E052A4C8
:10650000C5D852B4D5D8252EFAD71200420E4E6EF9
:10651000480E4D6E4A6A4B6A4C6A1200400E4E6E2F
:10652000490E4D6E0F0E4C6EDA0E4B6EA20E4A6E79
:106530001200400E4E6E130E4D6E5D0E4C6E8D0EA3
:106540004B6EDE0E4A6E12003F0E4E6E800E4D6E8A
:106550004A6A4B6A4C6A1200400E4E6E4A6A4B6A97
:106560004C6A4D6A1200410E4E6E200E4D6E4A6A04
:106570004B6A4C6A1200420E4E6EC80E4D6E4A6A4D
:106580004B6A4C6A1200440E4E6E7A0E4D6E4A6A89
:106590004B6A4C6A1200460E4E6E1C0E4D6E400E3B
:1065A0004C6E4A6A4B6A1200470E4E6EC30E4D6E19
:1065B000500E4C6E4A6A4B6A1200490E4E6E740EB3
:1065C0004D6E240E4C6E4A6A4B6A12004B0E4E6E94
:1065D000180E4D6E960E4C6E800E4B6E4A6A12006F
:1065E0004C0E4E6EBE0E4D6EBC0E4C6E200E4B6EA3
:1065F0004A6A12004E0E4E6E6E0E4D6E6B0E4C6E53
:10660000280E4B6E4A6A12003D0E4E6ECC0E4D6E39
:10661000CC0E4C6ECC0E4B6ECD0E4A6E12003C0E64
:106620004E6E230E4D6ED70E4C6E0A0E4B6E3D0E07
:106630004A6E12003A0E4E6E830E4D6E120E4C6E66
:106640006E0E4B6E980E4A6E1200350E4E6E860E12
:106650004D6E370E4C6EBD0E4B6E060E4A6E12001E
:10666000300E4E6E890E4D6E700E4C6E5F0E4B6E80
:10667000410E4A6E12002B0E4E6E8C0E4D6EBC0EED
:106680004C6ECC0E4B6E090E4A6E12006CDF89EF19
:1066900030F071DF89EF30F076DF89EF30F07BDFAB
:1066A00089EF30F081DF89EF30F087DF89EF30F05C
:1066B0005ADF09EF31F05FDF09EF31F064DF09EFF6
:1066C00031F069DF09EF31F06FDF09EF31F075DF8D
:1066D00009EF31F0A4EC2EF003E128EC38F01200C1
:1066E000C6EC2CF002013F0E176F800E166F136B75
:1066F000146B156B000128DF46EC31F055EC2DF0E2
:10670000A5EC2CF021DF4CEC31F060EC2DF0E7EC47
:106710002CF008EC2DF009EC31F055EC2DF06BEC81
:106720002DF0C6EC2CF0280E256ED1EC2CF014DFE9
:106730004CEC31F04AEC2DF0E7EC2CF01EEC2DF097
:1067400089EC30F01EEC2DF089EC30F055EC2DF09A
:10675000DCEC2CF009EC31F09AEC2CF04CEC31F044
:106760009AEC2CF04E50495C0BE14D50485C08E12E
:106770004C50475C05E14B50465C02E14A50455C99
:1067800005E0254E03D0C6EC2CF0CFD7E5DE89EF2F
:1067900030F00201276B0001B3EC32F048D806E379
:1067A00058EC33F00201272B0001F6D793DFC1DE4E
:1067B00009EC31F079EC2CF027C22BF02B5206E0DB
:1067C0000FEC2FF07EEC30F04CEC31F012007ED864
:1067D00034AE14D039AE29D05AD83450395C0BE1DC
:1067E0003350385C08E13250375C05E13150365C9B
:1067F00002E13050355CD8B016D017D034BE02D08C
:1068000039BE11D044D83450395C0BE13350385C78
:1068100008E13250375C05E13150365C02E130501E
:10682000355CD8B002D0D89001D0D88012004ED8B4
:1068300034AE14D039AE29D02AD83450395C0BE1AB
:106840003350385C08E13250375C05E13150365C3A
:1068500002E13050355CD8B016D017D034BE02D02B
:1068600039BE11D014D83450395C0BE13350385C48
:1068700008E13250375C05E13150365C02E13050BE
:10688000355CD8B002D0D88001D0D8901200A4ECEA
:106890002EF003E187EC2CF00FD0D890A8EC2DF06F
:1068A000D8903332323231323032338EA9EC2EF07E
:1068B00003E18EEC2CF009D0D890A2EC2DF0D8900A
:1068C0003832373236323532388E120045C030F029
:1068D00046C031F047C032F048C033F049C034F010
:1068E0004AC035F04BC036F04CC037F04DC038F0E0
:1068F0004EC039F0120002D881EF2DF0CEEC37F007
:1069000037D8050E226E00EE35F020EE26F07AEC38
:106910002CF010EE30F0050E236E22C024F0235030
:10692000242624062406EF50E602F350DE26D9CFB3
:106930004FF0DACF50F0F450DE22E86ADE22242E47
:10694000FCD74FC0D9FF50C0DAFF232EE6D7EE5256
:1069500020EE26F0060E246E2250245EDE52242EF7
:10696000FDD7222ED6D7DBEC37F052B20BD812006F
:10697000529234AE02D015D8527239AE02D020D81D
:1069800052721200261E271E281E291E2A1E262A83
:10699000D8B4272AD8B4282AD8B4292AD8B42A2A7D
:1069A0001200301E311E321E331E341E302AD8B45F
:1069B000312AD8B4322AD8B4332AD8B4342A1200AF
:1069C000351E361E371E381E391E352AD8B4362AD3
:1069D000D8B4372AD8B4382AD8B4392A1200C8DF34
:1069E000CEEC37F07AEC2CF0050E226E00EE35F08E
:1069F000EE6605D0222EFCD7DBEC37F01200226ABF
:106A0000222AD89039BE1CD035363636373638363D
:106A100039363950345C0BE13850335C08E137507B
:106A2000325C05E13650315C02E13550305CE8E221
:106A30007AEC2CF0D890393238323732363235325F
:106A40003950345C0BE13850335C08E13750325C2C
:106A500005E13650315C02E13550305C0AE33550D7
:106A6000305E3650315A3750325A3850335A3950D6
:106A7000345AC1EC2DF0222EDDD777DF30C035F04F
:106A800031C036F032C037F033C038F034C039F09E
:106A900081EC2DF0DBEF37F0290E226E7AEC2CF032
:106AA0003950345C0BE13850335C08E13750325CCC
:106AB00005E13650315C02E13550305C0BE3355076
:106AC000305E3650315A3750325A3850335A395076
:106AD000345AD880BAEC2DF0D890A8EC2DF039506B
:106AE000345C0BE13850335C08E13750325C05E12F
:106AF0003650315C02E13550305C0BE33550305E8E
:106B00003650315A3750325A3850335A3950345A35
:106B1000D880222EDFD71200CEEC37F0529234AE5E
:106B200002D03FDF52827AEC2CF0280E226E0A0E41
:106B3000236E00EE26F0EF500F0B246E050E245C42
:106B4000D8A002D0030EEF26EF50F00B246E500EAB
:106B5000245CD8A002D0300EEF26EC52232EEBD7C7
:106B6000D890A8EC2DF0BAEC2DF0222EE0D7DBEC7B
:106B700037F01200EBEC37F015E203EC38F01CE2D2
:106B80002FD844D85AD853941200030E4F6409D01A
:106B900050664F2A52B44F2A030E4F5E4F507CEC82
:106BA0000AF01200F2DF000EF86E580EF76EAE0E0D
:106BB000F66E8DEC0AF01200E8DF000EF86E580E4B
:106BC000F76EB20EF66E8DEC0AF01200EBEC37F0B9
:106BD000E9E203EC38F0F0E203D82FD85394120026
:106BE000CEEC37F000EE2FF012EE31F00A0E246EEC
:106BF000EDCF22F02238236E56D822C023F053D88E
:106C0000242EF6D7E76ADBEC37F01200CEEC37F033
:106C1000505210E002EE44F012EE44F0140E226ED8
:106C200050C023F0E5502206232EFCD7E5CFEDFF20
:106C3000222EFCD7DBEC37F01200CEEC37F00A0E38
:106C4000236E505023264F50235CD8B002D023C06F
:106C50004FF04F50505CD8A003D050C04FF04F2A97
:106C600050504F5E4F06090E226E4F50225E02EECC
:106C700031F0225204E0EECFE8FF222EFCD752A4DE
:106C800005D02B0E52BE2D0E92EC36F0528019D844
:106C9000529013D8505204E02C0E92EC36F009D8E2
:106CA000DBEC37F0120023500F0B3009E8CFE6FF82
:106CB000120050C024F0539606D0010E246E539655
:106CC00002D04FC024F0245226E052A006D0EFCFCD
:106CD00022F0300E225CD8A4529053A611D024C0CA
:106CE00030F0020E306202D08CEC36F0050E3062CD
:106CF00002D08CEC36F0080E306202D08CEC36F00C
:106D0000EECFE8FF52B003D092EC36F002D08EEC1A
:106D100036F0242EDAD71200200E04D0200E53B401
:106D2000300E00D0206E52A802D0010E546E546670
:106D300003D02050E7EC09F0010E546203D020503C
:106D4000BFEC0BF01200CEEC37F00A0E226E505062
:106D5000225E00EE26F0EF50224E0CD0EF50224E75
:106D600002D0EE52F8D7EE52306E490E306409D0A0
:106D7000010E06D00F0B306E040E306402D0100EE0
:106D8000EF260A0E226E00EE26F0EF500700EE6EA0
:106D9000E86AEF22222EF9D7DBEC37F01200CEECB6
:106DA00037F0050E226E0A0E236E00EE2FF0EDCFA7
:106DB00030F03050F00B07E1230630500F0B03E1A9
:106DC0002306222EF4D723C030F02350DBEC37F01B
:106DD000120032EC38F07AEC2CF08CEC35F026C056
:106DE0002BF027C02CF028C02DF029C02EF02AC08F
:106DF0002FF0050E4F6E506A52945394529853964A
:106E0000546A1200EBEC37F045E203EC38F042E252
:106E10005DEC30F052EC2EF026C000F227C001F2FB
:106E200028C002F229C003F22AC004F22BC030F0BD
:106E30002CC031F02DC032F02EC033F02FC034F012
:106E40008CEC35F026C007F227C008F228C009F202
:106E500029C00AF22AC00BF200C230F001C231F0A0
:106E600002C232F003C233F004C234F0EAEC2DF077
:106E700007C22BF008C22CF009C22DF00AC22EF076
:106E80000BC22FF0140E4F6E0A0E506E529853968E
:106E90005394546A52941200C6EC2CF0516A499EE5
:106EA000A4EC2EF014E0B3EC32F017EC34F001E077
:106EB00004E358EC33F0512AF6D7A4EC32F0E7ECB7
:106EC00033F005E004E346EC33F05106F6D702EC6C
:106ED00037F0A5EC2CF049BE528E0B0E4F6E0A0E09
:106EE000506E52845298546A1200E6EC35F0650EEA
:106EF00092EC36F0529E51BE528E51BE516C87ECD0
:106F00002CF051C030F0E9EC36F0528448DF30C04C
:106F10004FF0E6EC35F01200D1EC2CF09AEC2CF0AE
:106F200046EC31F076EC2DF0FDEC2CF0F2EC2CF090
:106F300046EC31F0BBEC2CF027C245F028C246F0FD
:106F400029C247F02AC248F02BC249F009EC31F0BF
:106F500076EC2DF013EC2DF0F2EC2CF046EC31F049
:106F600034EC2DF089EC30F09AEC2CF04CEC31F054
:106F70001200CEEC37F087EC2CF0050E226E10EEEE
:106F800026F020EE30F0E6500F0BDF6EE638F00B07
:106F9000DE12222EF8D7DBEC37F01200E9CF45F2F3
:106FA000EACF46F2E1CF47F2E2CF48F2D9CF49F239
:106FB000DACF4AF2120045C2E9FF46C2EAFF47C2F1
:106FC000E1FF48C2E2FF49C2D9FF4AC2DAFF12001C
:106FD00068EC30F003D05DEC30F000D0449E7F0EC2
:106FE00044620CD0800E436207D0426605D04166F1
:106FF00003D0406601D002D0D88001D0D8901200D2
:1070000068EC30F003D05DEC30F000D0449E7F0E91
:1070100044620BD0800E436208D0426606D04166BF
:1070200004D0406602D0D88001D0D890120002D897
:1070300073EF30F005D8448E120002D873EF30F0B1
:107040007F0E446E800E436E406A416A426A1200AF
:1070500002D873EF30F07F0E446E4068416842689A
:107060004368120002D873EF30F0406A416A426A06
:10707000436A446A1200410E4E6EA00E4D6E4A6A7B
:107080004B6A4C6A12003BEC38F009EC31F046ECEC
:1070900032F0C6EC2CF0A4EC32F04CEC31F04AECBF
:1070A0002DF0A5EC2CF0A4EC32F046EC31F0BBEC6A
:1070B0002CF0D1EC2CF009EC31F012004BC245F071
:1070C0004CC246F04DC247F04EC248F04FC249F0A4
:1070D00058EC33F046EC32F045C055F246C056F25B
:1070E00047C057F248C058F249C059F2120055C281
:1070F00045F056C246F057C247F058C248F059C250
:1071000049F05EEC33F086EC32F089EC30F0B5EC0F
:1071100031F045C060F246C061F247C062F248C03B
:1071200063F249C064F2120060C245F061C246F0E9
:1071300062C247F063C248F064C249F00201010E26
:10714000656F000125EC33F0E7EC33F009E3020151
:10715000040E656F000155EC33F04CEC33F018D0A1
:107160001AEC33F0E7EC33F007E30201030E656F2E
:10717000000155EC33F00CD0A4EC32F0E7EC33F026
:1071800007E30201020E656F00014CEC33F000D002
:1071900045C05BF246C05CF247C05DF248C05EF29B
:1071A00049C05FF2120055C245F056C246F057C2C0
:1071B00047F058C248F059C249F00201030E5A6F15
:1071C00000013BEC33F0E7EC33F00BE355EC33F02C
:1071D00055EC33F04CEC33F00201080E5A6F00010D
:1071E0004CD030EC33F0E7EC33F009E355EC33F0FE
:1071F00055EC33F00201070E5A6F00013ED025EC2A
:1072000033F0E7EC33F009E355EC33F04CEC33F0BA
:107210000201060E5A6F000130D01AEC33F0E7EC91
:1072200033F007E355EC33F00201050E5A6F00010D
:1072300024D0A4EC32F0E7EC33F007E34CEC33F06D
:107240000201040E5A6F000118D0DDEC32F017EC89
:1072500034F007E367EC33F00201010E5A6F0001CE
:107260000CD0C3EC32F017EC34F007E35EEC33F0F3
:107270000201020E5A6F000100D045C050F246C014
:1072800051F247C052F248C053F249C054F21200C2
:1072900050C245F051C246F052C247F053C248F0C6
:1072A00054C249F002EC37F0050E4F6E010E506EDD
:1072B000B3EC32F0E7EC33F003E3040E506E0FD082
:1072C000BBEC32F0E7EC33F003E3030E506E07D073
:1072D000C3EC32F0E7EC33F002E3020E506E67D8F5
:1072E000A3EC36F0E6EC35F05AC230F0030E306213
:1072F00009D0000EF86E580EF76EB60EF66E8DECD5
:107300000AF054D0040E306209D0000EF86E580E08
:10731000F76EBA0EF66E8DEC0AF048D0050E3062AC
:1073200009D0000EF86E580EF76EBE0EF66E8DEC9C
:107330000AF03CD0060E306209D0000EF86E580EEE
:10734000F76EC20EF66E8DEC0AF030D0070E30628A
:1073500009D0000EF86E580EF76EC60EF66E8DEC64
:107360000AF024D0020E306209D0000EF86E580EDA
:10737000F76ECE0EF66E8DEC0AF018D0010E30626C
:1073800009D0000EF86E580EF76ED20EF66E8DEC28
:107390000AF00CD0080E306209D0000EF86E580EBC
:1073A000F76ECA0EF66E8DEC0AF000D01200CFEC2C
:1073B00036F0030E306402D0010E506E030E3062C0
:1073C00002D0020E506E020E306202D0030E506EDA
:1073D000010E306202D0040E506E000E306202D0F8
:1073E000040E506E12005BC245F05CC246F05DC2F6
:1073F00047F05EC248F05FC249F002EC37F0060E7B
:107400004F6E010E506EC3EC32F0E7EC33F002E346
:10741000020E506EBBEC32F0E7EC33F002E3030EE9
:10742000506EB3EC32F0E7EC33F002E3040E506E32
:10743000BEDFA3EC36F0E6EC35F065C230F0010EAD
:10744000306209D0000EF86E580EF76ED60EF66E4A
:107450008DEC0AF024D0020E306209D0000EF86ED6
:10746000580EF76EDA0EF66E8DEC0AF018D0030E99
:10747000306209D0000EF86E580EF76EDE0EF66E12
:107480008DEC0AF00CD0040E306209D0000EF86EBC
:10749000580EF76EE20EF66E8DEC0AF000D0120078
:1074A0004BC245F04CC246F04DC247F04EC248F0C8
:1074B0004FC249F002EC37F0050E4F6E020E506ECF
:1074C000A3EC36F0CFEC36F0030E306004D0040E9F
:1074D0004F6E020E506E020E306404D0040E4F6EDA
:1074E000010E506E24D04BC245F04CC246F04DC246
:1074F00047F04EC248F04FC249F002EC37F0040E9C
:107500004F6E010E506EA3EC36F0CFEC36F0030E4A
:10751000306004D0030E4F6E010E506E020E3064C8
:1075200006D0040E4F6E000E506EA3EC36F052845F
:10753000E6EC35F0000EF86E580EF76EE60EF66EBD
:107540008DEC0AF0120050C245F051C246F052C212
:1075500047F053C248F054C249F002EC37F0040E31
:107560004F6E010E506EB3EC32F0E7EC33F003E3F4
:10757000030E506E0FD0BBEC32F0E7EC33F003E3B8
:10758000020E506E07D0C3EC32F0E7EC33F002E3AA
:10759000010E506EA3EC36F065D8E6EC35F05AC219
:1075A00030F0030E306209D0000EF86E580EF76E00
:1075B000B60EF66E8DEC0AF054D0040E306209D08F
:1075C000000EF86E580EF76EBA0EF66E8DEC0AF0DD
:1075D00048D0050E306209D0000EF86E580EF76ED6
:1075E000BE0EF66E8DEC0AF03CD0060E306209D06D
:1075F000000EF86E580EF76EC20EF66E8DEC0AF0A5
:1076000030D0070E306209D0000EF86E580EF76EBB
:10761000C60EF66E8DEC0AF024D0020E306209D050
:10762000000EF86E580EF76ECE0EF66E8DEC0AF068
:1076300018D0010E306209D0000EF86E580EF76EA9
:10764000D20EF66E8DEC0AF00CD0080E306209D026
:10765000000EF86E580EF76ECA0EF66E8DEC0AF03C
:1076600000D01200CFEC36F0030E306404D0050ECB
:107670004F6E000E506E030E306202D0010E506E3F
:10768000020E306202D0020E506E010E306202D045
:10769000030E506E000E306202D0030E506E1200C8
:1076A00050C245F051C246F052C247F053C248F0B2
:1076B00054C249F002EC37F0030E4F6E010E506ECB
:1076C000B3EC32F0E7EC33F003E3020E506E11D06E
:1076D000BBEC32F0E7EC33F003E3010E506E09D05F
:1076E000C3EC32F0E7EC33F004E3000E506E040E0E
:1076F0004F6EA3EC36F065D8E6EC35F05AC230F0A8
:10770000030E306209D0000EF86E580EF76EB60EFA
:10771000F66E8DEC0AF054D0040E306209D0000EE3
:10772000F86E580EF76EBA0EF66E8DEC0AF048D071
:10773000050E306209D0000EF86E580EF76EBE0EC0
:10774000F66E8DEC0AF03CD0060E306209D0000EC9
:10775000F86E580EF76EC20EF66E8DEC0AF030D051
:10776000070E306209D0000EF86E580EF76EC60E86
:10777000F66E8DEC0AF024D0020E306209D0000EB5
:10778000F86E580EF76ECE0EF66E8DEC0AF018D02D
:10779000010E306209D0000EF86E580EF76ED20E50
:1077A000F66E8DEC0AF00CD0080E306209D0000E97
:1077B000F86E580EF76ECA0EF66E8DEC0AF000D019
:1077C0001200CFEC36F0030E306404D0040E4F6E7E
:1077D000000E506E030E306204D0040E4F6E000E89
:1077E000506E020E306202D0010E506E010E3062F9
:1077F00002D0020E506E000E306202D0020E506EA9
:02780000120074
:020000040030CA
:0300010002191EC3
:02000500018078
:0200000400F00A
:10000000010107BCCBB3C83B5DCC0D84C2638C310E
:09001000C63BE79CF383C2162EE7
:00000001FF
